:10000000C8C200000C949032E1C20000DFC20000C0
:10001000DDC20000DBC20000D9C20000D7C2000070
:10002000D5C20000D3C200000C94C6300C94AE318F
:100030000C947B30CBC20000C9C20000C7C20000D4
:10004000C5C20000C3C20000C1C20000BFC20000A0
:10005000BDC200000C94A230B9C20000B7C20000BB
:10006000B5C20000B3C20000B1C20000AFC20000C0
:10007000ADC20000ABC20000A9C20000A7C20000D0
:10008000A5C20000A3C20000A1C200009FC20000E0
:100090009DC200009BC2000099C2000097C20000F0
:1000A00095C2000093C2000091C200000501090240
:1000B000A10185020901A1000509190129081500FE
:1000C0002501950875018102050109300931158165
:1000D000257F95027508810609381581257F9501D0
:1000E00075088106050C0A38021581257F95017572
:1000F000088106C0C005010980A101850319012AF4
:10010000B700150126B700950175108100C0050CD8
:100110000901A101850419012AA002150126A002E6
:10012000950175108100C00660FF0961A101096297
:10013000150026FF00952075088102096315002629
:10014000FF00952075089102C005010906A101056F
:100150000719E029E7150025019508750181029529
:1001600001750881010507190029FF150026FF0008
:100170009506750881000508190129051500250156
:10018000950575019102950175039101C00000006C
:10019000000000000000000000000000000000005F
:1001A000000000000000000000000000000000004F
:1001B000007E0F00D4FFFFFFC700000078000000A2
:1001C00000000000002A2B280000000000000000B2
:1001D000000000000000000029000000002C1E3478
:1001E00020212224342627252E362D3738271E1F7E
:1001F000202122232425263333362E37381F0405A9
:10020000060708090A0B0C0D0E0F10111213141516
:10021000161718191A1B1C1D2F3130232D350405F4
:10022000060708090A0B0C0D0E0F101112131415F6
:10023000161718191A1B1C1D2F3130354C09025B7B
:1002400000030100A0FA09040000010301010009F4
:100250002111010001224400070581030800010962
:100260000401000203000000092111010001222203
:100270000007058203200001070503032000010990
:100280000402000103000000092111010001227B8A
:10029000000705840320000112010002000000088D
:1002A000EDFE2CF20100010203011C03760069003F
:1002B00061006C003A0066003600340063003200D2
:1002C0006200330063000000180346006F007200F4
:1002D000200053006300690065006E006300650044
:1002E00000000A035000650065006A000000040376
:1002F00009042B00290026022F022F0014001A00E7
:1003000008001500170004221600070009000A0063
:100310001D221B4106001900050000000000E0003E
:10032000E300E20030003002270234002A001C0003
:1003300018000C00120013000B000D000E000F003F
:100340002800110010003600370038412C4121529E
:10035000E500000000003502350036022D022D00B8
:100360001E001F002000210022003A223B003C001A
:100370003D003E003F22404141004200430000005A
:1003800000000100010001002E022E0037023100A2
:100390004C00230024002500260027004B004A00C3
:1003A00052004D0033004E00500051004F0001003C
:1003B000235201000100000000003502010001008D
:1003C000010001002B0001000100010001000100FB
:1003D0000100010001000100010001000100010015
:1003E00001000000000001000100010014000100F4
:1003F00001000100010001000100010001000100F5
:1004000001000100010001000100010001000100E4
:100410000100010001000100010000000000007C5B
:100420000100010001000F080100010001000100AE
:1004300001000100010001000100010001000100B4
:1004400001000100010000000000010001000100A6
:100450001409010001000100057001000100010004
:100460000100010001000100010001000100010084
:100470000100010001000100010001000100000075
:100480000000FD377A585A000004E6D6B446020050
:10049000210116000000742FE5A3E00192009F5D8A
:1004A000003D8889A654750A36E182AEFA7A1AA60A
:1004B000FCA2ED4946CE36BE5D4D42F73F1400C367
:1004C00016CC1006C5BBA01569F43B3618718C52CA
:1004D0007E8DD09F54BADDD8FDF1DF6AA236ED766D
:1004E0001B84DA0E735A61428ABDC145CD13C1A285
:1004F0004A5429774C61C838184B3ED23D8AB9B569
:10050000C7E247714D35AB44BA5AB75B3E4BDB048B
:100510002494119120E9F20714E154B28C59B111DD
:100520003F7205ADCCE956ABD6BA8019F009185622
:100530008AFA0B0003DFF76F8A08B1B5DF3B35009D
:100540000000D0DEC12FCA7B872B0001BB019303C3
:100550000000C8EE8B23B1C467FB0200000000045A
:10056000595A504F52514A4D4B4E2A4C2F30B6B724
:10057000ABACBBBCA9AABDBECFD0CDCEDBDCD9DA3B
:100580000D0E0B0F1A0508050905071811130408AD
:10059000120C11241FBECFEFDAE0DEBFCDBF11E099
:1005A000A0E0B1E0EEE3FAE602C005900D92AC3BAC
:1005B000B107D9F725E0ACEBB1E001C01D92A3353E
:1005C000B207E1F70E9426290C94A13419CD9C01B1
:1005D0009A9581159F4118F5F32FF270EE27832F1E
:1005E0008170732F74706627532F5870442734FF1F
:1005F0000CC08295807FEF2B09F08062672B09F099
:100600008064452B69F080680895EF2B09F08260C3
:10061000672B09F08460452B19F08860089580E00D
:100620000895CF93DF93EB01D2DFFE010995DF91AF
:10063000CF9108950C94EF330895982F92959F7061
:1006400024E0911102C020E0982F892F869586958D
:10065000811511F02E5F982F892F8695820F0895AE
:1006600080934F05089580935005089521E030E070
:1006700001C0220F8A95EAF780915005822BF3CFB3
:1006800021E030E0A90102C0440F551F8A95E2F72E
:10069000CA018095909150058923E5CF292F9A3082
:1006A00090F5853080F590E035E0239F800D911D19
:1006B0001124282F277041E001C0440F2A95EAF742
:1006C00023E0969587952A95E1F7FC01EE0FFF1F31
:1006D000E80FF91FE150FD4F20E030E070E051914C
:1006E000DF01CB01022E02C0969587950A94E2F7AE
:1006F000817081958527842385278E932F5F3F4FB7
:100700002330310561F70895292F9A3078F5853027
:1007100068F590E035E0239F800D911D1124682F2E
:10072000677023E0969587952A95E1F7FC01EE0F17
:10073000FF1FE80FF91FE150FD4F40E050E080E05F
:10074000219130E0062E02C0369527950A94E2F7F3
:1007500021703327042E01C0220F0A94EAF7822B5E
:100760004F5F5F4F4330510559F7089580E008957A
:100770009091500521E030E0F90101C0EE0F8A951B
:10078000EAF7D90102C0AA0FBB1F6A95E2F7EA2B6C
:1007900001C0220F4A95EAF7892F8E23E81303C080
:1007A000892F822B60CF2095822F8923FBCF8091C8
:1007B000AD029091AC02981301C008958F5F8770CD
:1007C000FACF90919B048095892380939B04282FD6
:1007D0002770211110C0891771F09091520592FF76
:1007E0000AC08695869586954BDF10929B041092E1
:1007F0009D0410929C04089590919804982B9093D6
:1008000098040895982F9095809198048923809357
:100810009804089580919704811531F010929704FF
:1008200010929F0410929E040895803E9105D9F184
:10083000C8F48133910509F482C048F489329105E6
:1008400009F472C08A32910509F480C00895893391
:100850009105E9F082389105D1F08533910509F4CD
:100860005EC00895843E9105D9F148F4823E910519
:1008700039F1833E910549F181EE90E00895863E7D
:100880009105C9F1873E910509F43EC00895209174
:1008900051052370211164C02091520523FF14C01B
:1008A00089E290E008952091510520FD45C03091E6
:1008B000520530FF09C024FD24C083EE90E0089566
:1008C0002091510522FDF7CF08952091510522FD79
:1008D00044C03091520530FD43C024FFF5CF11C014
:1008E0002091520521FFF0CF8091510584FD09C070
:1008F00087EE90E008952091510523FFE5CF24FF76
:10090000F7CF80E090E008952091510523FD2BC0A2
:100910003091520531FFE1CF84EE90E008952091AF
:10092000510525FFD1CFBCCF2091510525FD1EC01B
:100930002091520523FFC8CF89E390E008952091CC
:10094000510526FFC1CF8AE290E00895209151051C
:1009500026FFBACF81E390E0089582EE90E00895FB
:1009600080EE90E0089586EE90E0089585E390E0B3
:1009700008959091510592FF10C041E0282F2471F5
:10098000243009F040E031E0282F2871283009F0A8
:1009900030E0431711F02CE0822793FF10C041E0B4
:1009A000282F2471243109F040E031E0282F2871EC
:1009B000283109F030E0431711F02CE08227309104
:1009C000520530FF10C051E0282F2171213009F06D
:1009D00050E041E0282F2871283009F040E05417FA
:1009E00011F029E0822731FF10C041E0282F21714A
:1009F000213109F040E031E0282F2871283109F039
:100A000030E0431711F029E0822794FD877E089596
:100A10001F93CF93DF9309DFEC01811522E5920745
:100A200008F052C0811540E5940708F0CDC0803E23
:100A3000910520F58D3C910508F0A1C0883A9105FB
:100A400070F4853A910508F097C081309105B9F1AD
:100A50000497813A910598F1C0E0D0E030C0885AFF
:100A600091094B97C8F7C85AD0E0CC0FDD1FC15B86
:100A7000DE4F0990D881C02DD46421C0811550E487
:100A80009507B0F4C11580E2D80708F0B3C0C83E9E
:100A9000D105A8F0CE019A9581159F41E8F68D2FDA
:100AA00068DF182FCE019927C0DEEC01D12B07C0DB
:100AB0009927BBDECC27DF70C82BD92BD06ACE019B
:100AC000DF91CF911F910895803842E59407C8F5D2
:100AD000803652E5950708F05BC0C03482E5D80740
:100AE000D0F4C03292E5D90708F04BC08C2F869520
:100AF000869520E2829FC0011124C37021E030E07E
:100B0000A90102C0440F551FCA95E2F7EA01C82B9C
:100B1000D92BDD68D4CF8C2F86958695877050E2CF
:100B2000859FC0011124C37021E030E0A90102C0FB
:100B3000440F551FCA95E2F7EA01C82BD92BDC6890
:100B4000BECF803C52E5950758F48F71C03AD2452C
:100B5000A0F590E0982F8827EC01C46FD06AAFCF42
:100B6000805C9245809708F077CFDC2FCC27CC278C
:100B7000DF71C06FD06AA3CFA497D064A0CFD06537
:100B80009ECFCF71D0E0DC2FCC27C16FD06A97CF3A
:100B900086958695877020E2829FC0011124C370DC
:100BA00021E030E0A90102C0440F551FCA95E2F7C9
:100BB000EA01C82BD92BDA6882CFDBDEC82FD0E060
:100BC000DC2FCC27D0627BCF8F71D3DE93E0CC0FAC
:100BD000DD1F9A95E1F7CC27DF70282F30E084FFE6
:100BE00005C050E1859F900111243327C22BD32BE0
:100BF000D06965CF8D2F8F71BCDE182FCE0199275C
:100C000014DEEC01D12BDECF80E00895F894E82FBC
:100C1000E295EF70F0E041A18F7021E030E0B90182
:100C200002C0660F771F8A95E2F7CB01962F909549
:100C3000942391A392A1892B82A37894089581157E
:100C40002CE7920741F420917C0230917D02232B06
:100C500011F480E090E00895E0E1F4E080E090E0BD
:100C600063EE77E246E058E228E738E2778366836E
:100C700051874087338722879787868701967096AA
:100C80008830910599F70895FB01811520E29207BC
:100C900028F4811541E0940738F408959C013052FE
:100CA0002115304348F00895392F94FF02C0329542
:100CB000307F2081232B208399270895462B22FF04
:100CC0000FC0982F92959F708F70892B962F9295B9
:100CD0009F706F70692B942F92959F704F70492B66
:100CE000982F9623961309C050E04095509590E0B8
:100CF0004823592381E0452B09F080E008951092A4
:100D0000E1041092E004E0EAF4E08581811102C080
:100D100014821682379684E0E83DF807B1F708950B
:100D2000AC013091E3046091E204232F621301C00F
:100D30000895822F90E0FC01EE0FFF1FE852FB4F59
:100D40000190F081E02DE417F50791F467E0649FCE
:100D5000F001659FF00D1124E056FB4F41E0448304
:100D60002313E6CF0196837099278093E3040895B7
:100D70000196282F2370DACFFC018481862381110C
:100D80000AC082818115B9F06823908593FF05C060
:100D900081E061110FC080E00895282F22952F7007
:100DA0008F70282B962F92959F706F70962B81E0F5
:100DB0002913F1CF089581E008950F931F93CF93E6
:100DC00001E010E0082E01C0000F0A94EAF7C0917C
:100DD00096049C2F9023911115C090919B04969599
:100DE00096959695891306C010929B0410929D04C7
:100DF00010929C043BDCC027C0939604CF911F91B6
:100E00000F9108953DDCF7CF282F35EB2303C00168
:100E1000112497FF04C080589109892F08958058A4
:100E20009F4FFBCF8091160380FD14C081FD14C03D
:100E300082FD16C080911503811581F08E3180F4FA
:100E400020E5829FC00111246EE170E00E94D6333C
:100E5000862F089584E1089588E2089588E0089532
:100E600080E508958091160380FD17C081FD17C0AD
:100E700082FD19C080911403811599F0883298F48D
:100E800028E0829FC001112468E270E00E94D633FE
:100E90006115710551F0862F089562E0FCCF64E082
:100EA000FACF61E0F8CF68E0F6CF81E00895909145
:100EB000720389029001112437FF03C080937203EB
:100EC00008952F3731051CF4980F909372030895FD
:100ED0009C0180E090E0F901E80FF91FE491E41330
:100EE00007C091E08927F901E80FF11D8491089569
:100EF0000196861780F380E00895FA01309709F093
:100F00000995089580919602811569F0E091A202F9
:100F1000F091A302309739F00190F081E02D3097E5
:100F200011F00995089580E00895A3E0B0E0EBE9A1
:100F3000F7E00C94AF339C018091EC019091ED01AE
:100F400082179307B1F03093ED012093EC01E0910B
:100F5000A202F091A302309761F00084F185E02DA8
:100F6000309739F083E089833B832A83CE01019651
:100F700009952396E2E00C94CB33A3E0B0E0E3ECD8
:100F8000F7E00C94AF339C018091EA019091EB0162
:100F900082179307B1F03093EB012093EA01E091BF
:100FA000A202F091A302309761F00084F185E02D58
:100FB000309739F084E089833B832A83CE01019600
:100FC00009952396E2E00C94CB339C01FC01329608
:100FD0008FEF90E04191461751F08F3F19F4411186
:100FE00001C0892F9F5F9630A9F78F3F09F40895BC
:100FF000280F311D87FD3A95F90162830895E0ECD1
:10100000F1E09191891302C0DF011E9291E0E63C6C
:10101000F907B9F708958091010108952FB7F89461
:101020008091E6019091E701A091E801B091E9017A
:101030002FBF0895962F2091520522FF0EC0682FD2
:10104000660F660F660F692B60939B040FDBE6DF6C
:1010500090939D0480939C04089508CB90919704ED
:10106000292F2823211559F08095892380939704EF
:10107000811531F0D3DF80939E0490939F040895EF
:1010800080E090E0F8CFCADF2091190330911A0375
:10109000232B211521F080936B0290936C022091F9
:1010A0001B0330911C03232B211521F0809369022F
:1010B00090936A02E091A202F091A302309759F056
:1010C0000680F781E02D309731F082E0809317039E
:1010D00087E193E009950895611509F441C0E3E3C0
:1010E000E80FE33148F4F0E0ED55FB4C0C94E933A4
:1010F00099DE819580931A03C6CF94DEFBCF92DEF2
:10110000819580931903F8CF8DDEFBCFABDE809302
:101110001B03F2CFA7DE8195FACFA4DE81958093E1
:101120001C03EACF9FDEFBCF815D990B21E030E00D
:1011300001C0220F8A95EAF780911803822B8093D1
:101140001803DACF80911603816080931603D4CF01
:10115000809116038260F9CF809116038460F5CFE9
:10116000409119038D3C59F480911A0387FF0DC0FB
:1011700010921A03411559F41092150308C08E3CC1
:1011800081F480911A0318169CF3411581F0809127
:101190001B0390911C03892B8111AECF1092140375
:1011A000ABCF8F3C41F447FFF0CF109219038091F1
:1011B0001A038115E0CF803D19F41416B4F3E5CF7E
:1011C00090911B03893D29F41916FCF610921B031C
:1011D000DCCF8A3D19F497FFD8CFF8CF90911C034C
:1011E0008B3D29F497FFD1CF10921C03CECF8C3DBD
:1011F00019F41916CCF3C9CF9FE2980F983090F4E8
:10120000815D990B21E030E0B90102C0660F771FC4
:101210008A95E2F7CB0180959091180389238093FA
:101220001803B3CF8D3D31F4809116038E7F8093E8
:101230001603ABCF8E3D21F4809116038D7FF7CF3F
:101240008F3D09F0A2CF809116038B7FF0CF2FB78F
:10125000F8946091E6017091E7018091E801909126
:10126000E9012FBF08950F931F9380919602811576
:1012700021F0EDDF1F910F910895E9DF00919802B1
:101280001091990220919A0230919B02600F711F78
:10129000821F931FEFCFCF92DF92EF92FF92CF93F7
:1012A000DF93D82FC92FC0900A04D0900B04E09090
:1012B0000C04F0900D04CBDF6C197D098E099F0999
:1012C000643F71408105910510F1C1DF6B017C0124
:1012D00082E390E0A0E0B0E0C0926502D0926602A6
:1012E000E0926702F092680280936102909362023A
:1012F000A0936302B0936402D0930804C0930904DE
:10130000DF91CF91FF90EF90DF90CF90089584EF21
:1013100091E0A0E0B0E0E0CF87E797E79093010885
:101320008093000888E19AE00FB6F894A89580931E
:1013300060000FBE90936000FFCF0895FC019B01F9
:101340008091DC019091DD018617970740F0672BB3
:1013500029F48091E8008E778093E800C90140E08D
:10136000009741F4411106C08091E80082FF2FC030
:1013700080E0089520917E022115A9F12530A9F180
:101380002091E80023FD2DC02091E80022FDECCF44
:101390002091E80020FFE4CF3091F3002091F2008B
:1013A000009719F02830310558F041E02830310518
:1013B00009F040E02091E8002E772093E800D0CF9C
:1013C00041914093F10001972F5F3F4FE9CF80910A
:1013D0007E02811541F0853041F08091E80083FF65
:1013E000C3CF81E0089582E0089583E0089580915D
:1013F000D60187FF13C08091E80082FF06C080916C
:10140000E8008B778093E800089580917E02811137
:10141000F2CF089580917E028115D9F38091E80082
:1014200080FFF8CF8091E8008E77ECCF2091E40028
:101430003091E50095E6A9012091EC00822F8170A2
:1014400020FF06C08091E80080FF06C080E008957C
:101450002091E80022FD1AC080917E02811589F05A
:10146000853089F08091EB0085FD0FC02091E4006C
:101470003091E50042175307F9F29A95E1F684E0BE
:10148000089582E0089583E0089581E00895E8EDED
:10149000F0E080818E7F80831092E2001092DA006B
:1014A0001092E100A0EEB0E08C9181608C9380817D
:1014B0008F77808319BCA7EDB0E08C918E7F8C93E1
:1014C00080818F7E80831092D5010895E091A202E1
:1014D000F091A302309739F00284F385E02D309724
:1014E00011F060E209950895FC01AC014B5F5F4F7C
:1014F0008FEF61E39191892728E030E0982F990FD1
:1015000087FF09C0892F862721503040B9F7E4179B
:10151000F50781F70895892FF7CF982F9093E90069
:10152000891771F07091EC002091ED005091F0005E
:1015300021FD09C09F5F973089F78093E9000895E6
:10154000762F242F50E03091EB003E7F3093EB005C
:101550003091ED003D7F3093ED003091EB00316034
:101560003093EB007093EC002093ED005093F0006B
:101570002091EE0027FDDECF0895A0E0B0E0E3EC7F
:10158000FAE00C94A933C8EDD0E088818F7E88837F
:10159000E7EDF0E080818160808384E082BF81E0BC
:1015A0008093D50188818E7F888302EE10E0F80158
:1015B00010821092DA0081EEC82ED12CF601108232
:1015C00088818F77888388818068888388818F7DF0
:1015D000888319BC10927E021092D4011092550299
:1015E0001092D30190EEE92EF12CF70180818B7FD0
:1015F000808388818160888342E060E080E08DDFC5
:10160000F60180818E7F8083F801808181608083F4
:10161000808188608083F70180818E7F80838881CC
:1016200080618883CDB7DEB7E8E00C94C533E091E4
:10163000AD029091AC0229E0E91302C080E0089568
:10164000AE2FB0E02E9FF0011124E255FD4F318105
:10165000361306C03081381303C03581341304C0FB
:10166000FD013196E770E8CF81E008950F931F9355
:10167000CF93DF938B01EA0190917E02943051F574
:101680008093E9008FEF9091E80095FD06C095EDFD
:101690009A95F1F700008A95B1F78091E80085FFEF
:1016A00019C0C4DE811111C08091E80085FD06C01B
:1016B0008091E8008E778093E800F3CFF801819164
:1016C0008F018093F100219779F78091E8008E7760
:1016D0008093E800DF91CF911F910F910895792FAA
:1016E000603229F440E250E0682F82E0BFCF0895D5
:1016F000CF93DF93D82FC92F48E050E0682F792F80
:1017000081E0B4DF88E0ED2FFC2FAEEDB1E0019079
:101710000D928A95E1F7DF91CF910895BC0146E0E3
:1017200050E084E0A3CFBC0143E050E084E09ECFD2
:10173000A0E0B0E0EEE9FBE00C94A733F82EE92E30
:10174000B62EA72E8A018091D0019AE0C92ED12C05
:101750008A3018F0CC24C394D12CC1E0D0E06B2D9A
:101760007A2D8F2D9E2DF8010995811116C0219695
:10177000CC16DD0694F0CC9FC001CD9F900D900D4E
:10178000112420E030E045E34A95F1F700002F5F97
:101790003F4F28173907B9F7E2CFCDB7DEB7EAE0F8
:1017A0000C94C3339091520592FB222720F92817FD
:1017B00079F080FB92F990935205609151057091F8
:1017C000520584E090E00E94863482E00C94E103AC
:1017D00008951F93CF93DF93962F122F632F84309A
:1017E000D8F49A30C8F44530B8F4C42FD0E0CC0F08
:1017F000DD1F2AE0929FC00DD11D112494E6899F20
:10180000C00DD11D1124CE0189960E946C34612F28
:10181000CE018A960E946C34DF91CF911F9108957A
:10182000CF93DF93C091980480919A04C82B809144
:1018300097048115F1F0F2DB20919E0430919F0412
:10184000821B930B8838934110F00E940A04D091B8
:10185000970420E080EC91E0FC0130810196311189
:101860002F5F31E0863C9307B9F721110E940A04EB
:10187000CD2B80918C0380958C2390918B03892BA9
:101880008093BE0148E050E064EA72E08EEB91E0A4
:101890000E942334892BB9F088E0EEEBF1E0A4EA52
:1018A000B2E001900D928A95E1F7E091A202F091E9
:1018B000A302309741F00280F381E02D309719F0B8
:1018C0008EEB91E00995DF91CF910895CF9310921F
:1018D0009804C6E0E0ECF1E0DF018C2F1D928A95C0
:1018E000E9F780E090E021DB80E090E046DB1092B9
:1018F0009A0496DFE7E1F3E0DF011D92CA95E9F76C
:10190000109215031092140310921603BCDBCF91B2
:101910000895DCDF2FEF84E39CE02150804090406D
:10192000E1F700C0000088E19AE00FB6F894A895AE
:10193000809360000FBE90936000FFCFAAE2B0E0FA
:10194000E4EAFCE00C94AE3386ED91E0FC010196F4
:101950002091F100208321E08E3D9207B9F780911C
:10196000D701893009F457C0C8F4823009F4B2C0F5
:10197000833009F482C0813081F18091E80083FFD7
:10198000E6C08091D6019091D7019A3008F0DFC06F
:10199000E92FF0E0EA54FB4C0C94E9338A3009F467
:1019A00089C08B3051F78091D601813231F7809117
:1019B000DA019091DB01892B01F78091E800877FA4
:1019C0008093E80014DD81E09091D801911101C06D
:1019D00080E0809302017ADFD0CF8091D601813AF6
:1019E00061F68091E800877F8093E8008091DA01BA
:1019F0009091DB01892B59F060E080E090E070E08D
:101A00009DDC8091E8008B778093E800B6CF68E09A
:101A10008EED91E0F4CF8091D601813209F0ADCF07
:101A20008091DA019091DB018D7F892B09F0A5CFA0
:101A30008091E800877F8093E8008091E80082FF32
:101A400017C09091F3008091F200029731F48091D9
:101A5000F100813011F0863021F48091F100809303
:101A600001018091E8008B778093E800C0DC85CF8E
:101A700080917E028111E1CF80CF8091D601813AA1
:101A800009F07BCF8091DA019091DB01892B09F07D
:101A900074CF8091E800877F8093E8008091E80010
:101AA00080FFFCCF809102018093F1008091E800DB
:101AB0008E77DACF8091D601813209F05ECF8091A6
:101AC000E800877F8093E80092DC8091D9018093C1
:101AD000000153CF8091D601813A09F04ECF809119
:101AE000E800877F8093E8008091E80080FFFCCFCA
:101AF00080910001D9CF803889F0823841F58091FA
:101B0000DA018F70873018F58093E9008091EB003F
:101B100085FB882780F91092E90006C08091550264
:101B2000880F9091D301892B9091E800977F909333
:101B3000E8008093F1001092F1008091E8008E7728
:101B400023C0811116C08091D801813009F18091A4
:101B5000E80083FF0AC08091E800877F8093E80057
:101B60008091EB0080628093EB00AA96E3E00C94F6
:101B7000CA33823061F78091D801811581F01092CB
:101B8000E9008091E800877F8093E80030DCDFCFB8
:101B900081E0933009F080E080935502F0CF80918E
:101BA000DA018F702FEF280F263088F68093E90036
:101BB0002091EB0020FFE3CF933031F48091EB00D4
:101BC00080628093EB00DBCF9091EB00906190936B
:101BD000EB0021E030E0A90102C0440F551F8A95B7
:101BE000E2F74093EA001092EA008091EB008860EF
:101BF000E8CF8111ACCF1091D8011F778091E3001D
:101C00008078812B8093E3008091E800877F809328
:101C1000E800EDDB8091E80080FFFCCF8091E300DD
:101C200080688093E30083E0111101C082E080931B
:101C30007E028DCF8058823008F089CF8091D80104
:101C40009091D9018C3D53E0950791F583E08A830B
:101C50008AE289834FB7F894DE01139620E03EE0D4
:101C600051E2E32FF0E050935700849120FF03C02E
:101C700082958F703F5F8F708A30C0F0895C90E0F2
:101C80008D939D932F5F243161F74FBF8091E800C2
:101C9000877F8093E8006AE270E0CE0101964EDB18
:101CA0008091E8008B778093E80051CF805DE7CF8B
:101CB000292F33272330310509F44EC078F5213020
:101CC000310509F488C08BE590E0EDE3F2E02230C5
:101CD000310509F03CCF2091E800277F2093E800F0
:101CE0002091DC013091DD018217930708F49C01FB
:101CF00040E02115310509F073C0411171C0809198
:101D0000E80082FDCDCF80917E02811549F28530B9
:101D100039F28091E80083FFF2CFC2CF8091DA01DF
:101D20009091DB012132310509F446C022323105A0
:101D300009F00DCF8330910508F009CFFC01EE0FBB
:101D4000FF1FE95CFE4F0190F081E02D8C5C9E4FFF
:101D5000DC018C9190E010C09C013327823021F18E
:101D60002330310568F4232BB9F4EEEEF2E0E49170
:101D70008E2F90E0EEEEF2E0009709F4E8CEABCFC4
:101D80002330310509F0E3CEEAEAF2E0E4918E2F48
:101D900090E0EAEAF2E0F0CFE2EEF2E0E4918E2F9A
:101DA00090E0E2EEF2E0E8CFE8ECF2E0E4918E2F92
:101DB00090E0E8ECF2E0E0CF8330910508F0C7CE88
:101DC000FC01EE0FFF1FE35CFE4F0190F081E02D60
:101DD00089E090E080CF82E190E0E8E9F2E07BCF1B
:101DE00080917E02811509F45BCF853009F458CFCC
:101DF0008091E80083FD54CF8091E80082FD7FCF81
:101E00008091E80080FF75CF9091F3008091F200FF
:101E10002115310519F08830910550F041E00897FF
:101E200009F040E08091E8008E778093E80061CF70
:101E300044914093F1003196215031090196E8CF49
:101E4000803809F084CE8091E800877F8093E80095
:101E50008091D4018093F10070CE811178CE1091E1
:101E6000D801123008F073CE8091E800877F80930C
:101E7000E8001093D401BBDA1115D9F084E0809307
:101E80007E0242E061EC81E048DB42E261EC84E00A
:101E900044DB42E261EC82E040DB42E260EC83E062
:101EA0003CDB80917E02843051F482E08093030118
:101EB0004ECE8091E30087FDE1CF81E0E0CF81E06D
:101EC000F5CFCF93C82F811599F08CEF8C0F813A05
:101ED00088F4E0ECF1E086EC91E02191C217B1F1D9
:101EE0008E179F07D1F76C2F8EEB91E06ED898DCA0
:101EF000CF91089580E28C0F883048F4C77081E05C
:101F000001C0880FCA95EAF70E94FC03F0CF8BE569
:101F10008C0F833030F42C2F2452330BC90105D899
:101F2000E7CFE8E5EC0FEB3148F4F0E0EE0FFF1FF0
:101F3000EB57FE4F8081918120D8DACF83E38C0F5D
:101F40008331B0F661E08C2FC7D8D2CF8C2F57D811
:101F500067DCC9CFCF93DF93EC01805E91090897CE
:101F600020F06EE070E1209711F462E070E1CE01A4
:101F70000E9411038C2FA5DFDF91CF910895811569
:101F800051F19CEF980F913A10F439D849CC90E276
:101F9000980F983050F4877091E001C0990F8A959E
:101FA000EAF7892F0E940204F1CF9BE5980F933046
:101FB00020F480E090E00C94950798E5980F9B3111
:101FC00020F480E090E00C94BD0793E3980F9331E8
:101FD00010F460E081C808951F93CF93DF93182F0A
:101FE000EB016FDF209731F4812FC9DFDF91CF91B3
:101FF0001F9108958FE99FE00197F1F700C000005D
:102000002197F0CF811519F00E94FC0309CC0895A7
:10201000811519F00E94020403CC0895811531F056
:1020200090919A04892B80939A04FACB0895811594
:1020300039F0809590919A04892380939A04F0CB8B
:10204000089580918703811521F082E2F0DF1092DC
:1020500087030895CF93DF93EC014A855B856E85F6
:102060007F850E947D079B81909580919A048923AA
:1020700080939A048C810E940204D2DB86E0FE01E8
:1020800011928A95E9F7DF91CF910895CF93DF936D
:10209000EC018D8181FD13C082608D8380919A0453
:1020A0009B81892B80939A048C810E94FC03B8DB6E
:1020B000488559856E857F85CE010E947D071092E7
:1020C0009104109290048D8180FD02C0CE01C2DF88
:1020D000DF91CF9108951F93CF93DF93182FA09195
:1020E0000604B0910704109709F448C0109209043F
:1020F0001092080410928C0310928B031696CD91C7
:10210000DC911797CE019A9581159F4108F4D07EF6
:10211000D1E0C11101C0D0E01996ED91FC911A9760
:10212000309731F01B966D917C9180E00995D82312
:10213000D11539F08CEF8C0F813A20F58C2F0E944D
:10214000FF071115A1F0E0910604F09107048085C6
:1021500084FD0DC080910504811549F08081918135
:102160009C01215031092F333E4708F494D858DBA5
:10217000109207041092060410920504DF91CF918B
:102180001F9108954DDB8C2FFADEDBCFAFE0B0E07E
:10219000ECECF0E10C94A633FE0131968AE0DF010D
:1021A0001D928A95E9F703E411E0BB24B3949E2EB7
:1021B000AF2EEE24E394F12C9DE4C92E91E0D92EAC
:1021C000F80181918F018F3F09F446C0F894E82F00
:1021D000E295EF70F0E021A18F70A70102C0440FDB
:1021E000551F8A95E2F7CA01922F982B91A392A1CD
:1021F0008095892382A3789400C0A8E4B1E0692D7A
:102200007A2D4B2D40959D91FB018191BF019F3F00
:1022100009F486C0292F22952F70205E30E0F90145
:10222000208130E09F7002C0359527959A95E2F79E
:1022300020FD76C08B299B0121503109F901808353
:10224000CA16DB0601F7F80182918F3F11F00E9458
:102250000606F0EAFA95F1F7BB0C21E00834120704
:1022600009F0AECF4AE050E0692D7A2D88E492E083
:102270000E9423349C01892B49F08AE0E92DFA2D34
:10228000A8E4B2E001900D928A95E1F70091530223
:1022900010E00E581D4F232B09F444C081E08093B9
:1022A000CF010E940E089093CE018093CD018091C2
:1022B0009602811509F490C07E014BE0E40EF11CFA
:1022C00085E0D7011D928A95E9F78091D0018A3087
:1022D00008F04CC049E253E1B701C80129DA811581
:1022E00009F468C04EEC52E1B701C80121DA81154A
:1022F00009F460C01092D0018091520290E045E054
:1023000050E0B7018E589D4F0E94233421E0209366
:10231000CC01892B09F041C02F96EBE00C94C2331D
:10232000842389CF8091CF01811509F4C0CFE0903B
:10233000CD01F090CE010E940E088E199F090597DD
:1023400008F4B5CF45E050E068E472E0C8010E94AF
:102350002334892B41F085E0E8E4F2E0D8010190D4
:102360000D928A95E1F71092CF01A1CFC090CA01DA
:10237000D090CB010E940E088C199D09843F91409A
:1023800008F0A8CF8091CC01811531F285E0F701EA
:1023900011928A95E9F71092CC01A0915202B0E017
:1023A000AE58BD4F85E0FE013B9601900D928A9597
:1023B000E1F7B2CF8091D0018F3F39F40E940E082F
:1023C0009093CB018093CA01DDCF8F5F8093D001C2
:1023D0008A3008F491CFF2CF85E0F801A4E8B2E0AA
:1023E00001900D928A95E1F784E892E07DD8809380
:1023F0008302C0908902D0908A02E0908B02F09014
:102400008C028091C6019091C701A091C801B09142
:10241000C901C816D906EA06FB0609F47DCFC092A9
:10242000C601D092C701E092C801F092C9010E9492
:102430002709C61AD70AE80AF90AC0929802D09268
:102440009902E0929A02F0929B0266CFA0E0B0E07F
:10245000ECE2F2E10C94A833EC018881811509F1DA
:10246000813009F045C08981813051F48A812396F9
:1024700060E570E0893311F060E070E0ADDDEDCF34
:10248000823021F48A8123961CDDE7CF833021F44A
:102490008A81239674DDE1CF843041F02296811148
:1024A000DCCFCDB7DEB7E9E00C94C4338A81239644
:1024B00020E030E09AE0682F6053770BAB016A3080
:1024C000710560F02115310551F3EFE9FFE0319717
:1024D000F1F700C0000021503109F4CF929FB00104
:1024E000939F700D11249A01260F371F8991E3CF16
:1024F000E82FF0E0E354FE4FB490282F2695269560
:10250000269530E0F901E355FE4FE4908770F12CF9
:10251000082E02C0F594E7940A94E2F7E0FAEE245C
:10252000FF24E0F8F901E356FE4FC490D12C082EA9
:1025300002C0D594C7940A94E2F7C0FACC24DD24F3
:10254000C0F8F901E357FE4F049110E002C0159561
:1025500007958A95E2F701701127E114F10411F053
:1025600081EEAFDCC114D10411F086EEAADC60E08C
:1025700070E08B2D31DDC114D10411F086EEFFDC4B
:10258000E114F10411F081EEFADC0115110521F0DE
:1025900060E070E08CE220DD21965FCFCF92DF9289
:1025A000EF92FF921F93CF93DF9300D000D0CDB76F
:1025B000DEB7C0907F02D0908002E0908102F09060
:1025C00082020E9427096C197D098E099F0911E07A
:1025D000643671058105910578F10E943309DC01AB
:1025E000CB010296A11DB11D89839A83AB83BC8365
:1025F00080912201909123018D579D4F20912101BF
:10260000422F50E0253010F044E050E0BE016F5FF3
:102610007F4F0E94303482E090E00E943133182FC7
:10262000811551F00E94270960937F027093800208
:102630008093810290938202812F0F900F900F90D0
:102640000F90DF91CF911F91FF90EF90DF90CF908F
:1026500008958F929F92AF92BF92FF920F931F9314
:10266000CF93DF9300D000D000D0CDB7DEB7F62EE9
:10267000072F80E090E00E943133182F811509F474
:1026800060C080911401482F50E0811511F041E0A5
:1026900050E060911501709116016D577D4FCE018C
:1026A00006960E9430348090920290909302A090FF
:1026B0009402B09095020E942709681979098A0945
:1026C0009B09643671058105910538F484E892E030
:1026D0000E94740A9E818917A1F181E090E00E9416
:1026E00031338115C9F180911C01482F50E08630AB
:1026F00010F045E050E060911D0170911E016D5792
:102700007D4FCE0101960E94303484E892E00E9411
:10271000740A9E81891320C00E9427096093920247
:1027200070939302809394029093950285E0FE014A
:102730003196ADE8B2E001900D928A95E1F781E023
:102740000CC085E0E4E8F2E0DE01119601900D9204
:102750008A95E1F71111EACF80E095E0EDE8F2E02B
:10276000AF2DB02F01900D929A95E1F70F900F9039
:102770000F900F900F900F90DF91CF911F910F91BD
:10278000FF90BF90AF909F908F9008950F931F93ED
:10279000CF93DF93843030F56A3020F5453010F563
:1027A000C42FD0E0CC0FDD1F2AE0629FC00DD11DE9
:1027B000112434E6839FC00DD11D1124CE018996CA
:1027C0000E945034082F10E0102F0027CE018A9667
:1027D0000E9450349801282BC901DF91CF911F919D
:1027E0000F91089580E090E0F8CF462F672F209159
:1027F0009E0230919F02232B81F4703F39F4403FB9
:1028000061F480919C0290919D0208957A3028F4A1
:10281000453018F4843008F4B9CF80E090E0089592
:10282000A0E0B0E0E6E1F4E10C94AA337C01009171
:10283000500580914F05082BC3E0D0E010E0C8019F
:102840000C2E02C0959587950A94E2F780FD09C089
:102850002197A8F7D12C8D2DCDB7DEB7E7E00C94EA
:10286000C633DC2EB7018C2FC0DF0E94080501970C
:1028700079F3F1CF0F931F93CF93FC01878190855C
:10288000009789F4858100811181811581F061159E
:1028900071F0C801C5DFC82F682FC8010E944E0320
:1028A000B8018C2FA2DFCF911F910F910895C8011D
:1028B0000E948403C82FF4CFCF93DF93D82FC92F62
:1028C000AFDF6D2F7C2F91DF0E940805DF91CF9144
:1028D0000895FC0184818115B1F08781908500976E
:1028E000A1F00E940805282F92959F709630B9F0AC
:1028F00080F4925F9F70923030F4203FD1F058F412
:1029000081E0283E58F080E0089580819181D4DFF5
:10291000EACF9A5FEFCF81E0243FA9F7089591E0D5
:10292000813F09F090E081E0283E08F080E0892BAB
:10293000089581E00895382F292FCB01A32FB22FBE
:10294000873221E09207A105B10520F487529D4FFF
:102950000C94503480E0089585E290E00E94503459
:10296000823A89F486E290E00E9450348D3A59F41C
:1029700087E290E00E94503491E08B3609F090E0BD
:10298000892F8170089580E0FCCFAAE0B0E0EBECE5
:10299000F4E10C94A433C0907C02D0907D0281E0DD
:1029A00090E090937D0280937C02812C912CE12C0D
:1029B0005401F12C15C0F80125913591472D6F2D4B
:1029C0008E2D0E94E90B0E5F1F4F739485E07812E5
:1029D000F2CF95E0A90EB11CF394EAE0FE1639F0AF
:1029E0008501000F111F0E501D4F712CE4CFE39491
:1029F000F2E38F0E911C84E0E812DACF1A8219827A
:102A00001C821B821E821D8218861F8288EC90E029
:102A10009A87898709EB11E0FE0131967F014AE030
:102A200050E0B801C7010E948A34065F1F4F093089
:102A3000F2E01F07A1F78AE0F70111928A95E9F702
:102A40004AE050E0B801C7010E948A34065F1F4F78
:102A50000935F2E01F07A1F789E0F70111928A9585
:102A6000E9F78FEF9FEF9E838D8387E08A874AE0A7
:102A700050E0B801C7010E948A34065F1F4F093A2F
:102A8000F2E01F07A1F786E0F70111928A95E9F7B6
:102A900046E050E0B801C7010E948A340A5F1F4F28
:102AA000093DF2E01F07A1F7D0927D02C0927C029F
:102AB0002A96EDE00C94C033AAE0B0E0E2E6F5E13E
:102AC0000C94A933E0EFF1E080E5DF011D928A95D7
:102AD000E9F7E0EAF4E088E3DF011D928A95E9F77F
:102AE00080EFC82E81E0D82E7F0109E012E0F701C7
:102AF000D182C0824AE050E0B801CE0101960E9426
:102B0000403488E0FE013196D60101900D928A95FD
:102B1000E1F789859A85D70113969C938E93129736
:102B2000BAE0CB0ED11CE7E0EE0EF11C065F1F4FA2
:102B30000935F2E01F07D9F62A96E8E00C94C53370
:102B4000AAE0B0E0E6EAF5E10C94A7330DE813E063
:102B500089E5E82E82E0F82E97E0B92E2FEEC22EFE
:102B600021E0D22EAA24A3944AE050E0B701CE017E
:102B700001960E944034F8013896DF018B2D1D929A
:102B80008A95E9F789819A81D80111969C938E9351
:102B90008F8112968C9312978D8113968C93139735
:102BA000888514968C931497898515968C93159720
:102BB0008B819C8117969C938E9316978A8587FDAF
:102BC00004C01E96DC92CE921D9780FF02C0F801D1
:102BD000A08681FF07C0D80118969C911897926033
:102BE00018969C9382FF04C0F801908594609087AA
:102BF00083FF07C0D80118969C9118979860189683
:102C00009C9384FF04C0F80190859061908785FFB4
:102C100007C0D80118968C911897806218968C93EB
:102C2000BAE0EB0EF11C015F1F4FE9EAEE16E2E09D
:102C3000FE0609F099CF2A96EAE00C94C333A6E089
:102C4000B0E0E5E2F6E10C94AA3307E213E089EA8A
:102C5000E82E82E0F82E98E0D92E46E050E0B70149
:102C6000CE0101960E944034F8018D2D11928A9573
:102C7000E9F7B8016C5F7F4F89819A810E94440611
:102C8000F80191838083B8016B5F7F4F8B819C81BA
:102C90000E944406F801938382838D8186838E810E
:102CA0008783F6E0EF0EF11C085F1F4F89EDE816F1
:102CB00082E0F80691F62696E7E00C94C633282FBA
:102CC000CB01283070F44AE0249F90011124B9010F
:102CD00067547E4F4AE050E00E94403480E090E02C
:102CE00008958FEF9FEF0895AAE0B0E0EAE7F6E1DC
:102CF0000C94AF339C0197558115914068F4BE0147
:102D00006F5F7F4F822FDBDF892B31F489859A85B6
:102D10002A96E2E00C94CB3388EC90E0F9CFA0E067
:102D2000B0E0E5E9F6E10C94AA33162FD72FC42FB3
:102D3000D22E8115A1F0409394040E940E08909326
:102D4000D2018093D101C77081E001C0880FCA957C
:102D5000EAF758D9CDB7DEB7E7E00C94C6339091C7
:102D60009404491335C0E090D101F090D2010E9443
:102D70000E089C012E193F097901812F9D2FB4DF88
:102D8000E816F90628F5D0E2DD0DCD1591F0C770F3
:102D900011E0812F01C0880FCA95EAF739D9D830E0
:102DA00040F48D2D877001C0110F8A95EAF7812FAD
:102DB00029D960E070E0802F0FD9D83058F62D2D3A
:102DC000277081E001C0880F2A95EAF721D9C2CF88
:102DD000C77081E001C0880FCA95EAF7F7CFACE071
:102DE000B0E0E5EFF6E10C949F337C01DC01149632
:102DF0008C91811509F4E8C061E0C7013BDD8C01CD
:102E0000F7018581811521F18091900490919104C1
:102E10000097F1F008171907D9F0FC01FF27887F08
:102E20009927892B09F04CC0B4E0EE0FFF1FBA952B
:102E3000E1F7E05FFB4F8581846085831183008328
:102E4000CF0124D910929A0461E0C70113DD8C01EF
:102E5000D70115969C9180917C03811138C0911502
:102E600009F469C00115B0E51B0708F050C0011551
:102E7000E0E21E0708F0ACC00115F7E01F0739F1CA
:102E800010F59801205E31092830310500F140919C
:102E9000980480919A043091970429E0F701A8E6FC
:102EA000B3E001900D922A95E1F71093700300931F
:102EB0006F0310927203842B832B8093670307C0E8
:102EC000E0E0F0E0B8CF01153FE0130701F7D09044
:102ED00098048D2D8D7D811531F082E0911509F4D6
:102EE00074C10E943603D70115964C91411509F41F
:102EF0004EC20A32110509F06BC18D2D8474811503
:102F000009F4F4C260E070E08CE466D84CC0003E86
:102F100042E5140748F4003652E51507C0F698015B
:102F2000325520343105B2CF980127573C47253020
:102F3000310508F0ACCF0937BCE71B0709F04DC0DD
:102F400020916F0330917003232B69F1911599F053
:102F500081E00E9457078091670360D889E0E8E626
:102F6000F3E0AEE1B3E001900D928A95E1F7809134
:102F7000720380931D0386E0F701AEE1B3E0019098
:102F80000D928A95E1F780911D0380937C038EE179
:102F900093E025DF10927C03F7018581811103C046
:102FA0008091670344D880919B048770811561F0FC
:102FB000D70115968C91811539F08091520582FFC9
:102FC00003C082E00E94E1032C96E2E10C94BB3343
:102FD000D70116968C91803159CF0A37FCE71F072D
:102FE00009F075CF911509F4C5C0A0906F03B0909A
:102FF0007003209167032D832983BE016F5F7F4F8C
:10300000C5010E9444062C0139813B87A7E2CA2EE4
:10301000A3E0DA2E01E010E022242A94D6011796CC
:103020003C90179733FE53C06D907C901197129689
:103030008D909C90139746145704B9F41496BC9144
:10304000B987232DF60146816B2F8B850E945E0682
:10305000811559F089850E941A03281634F4D60187
:1030600015969C918401192B282E48145904C9F4F3
:1030700031FE17C0F601F581F987232DD60116968A
:103080004C916F2F8B850E945E06811551F08985CA
:103090000E941A0328162CF4F60194818301192B3F
:1030A000282E30FE14C0FFEF2F1211C00130110581
:1030B00071F4232DD60116964C9160E08B850E9409
:1030C0005E06811521F0F60185818401182BF8E058
:1030D000CF0ED11C27E633E02C153D0509F09ECF1D
:1030E00001301105E1F58D8182958F703D81832B33
:1030F0008F7011E0303108F410E01295107F182B1A
:10310000A11440E2B40620F5A11451E0B50608F080
:1031100055C00A2D812F8D704A2D811509F451C09B
:103120006AE088E895E00E946807282F30E02115C2
:10313000310551F4402F6EE182E695E00E94680768
:10314000282F30E0811549F0F901F12B8F0107C0DC
:10315000C50190528115904390F100E010E087E0A6
:10316000E3E7F3E0DF011D928A95E9F710937B0313
:1031700000937A0380917A0390917B03892B09F461
:1031800012CFF7018581811539F08FEF0E94570723
:10319000809172038093710386E0F701A3E7B3E0A7
:1031A00001900D928A95E1F78091710380937C03E1
:1031B00083E793E014DE10927C03F5CE1B29BB2439
:1031C000A8CF68E080E895E0AECF0E9440038BCEA8
:1031D000C80197578038910508F068C1003108F0A0
:1031E000E2CE66E271E080E090E0A5DB8111DBCE0B
:1031F000812C912C5401011143C004E09E012F5FEA
:103200003F4F6901D601E02F1D92EA95E9F72401AD
:103210003501FFEF4F1A5F0A6F0A7F0AC501B4013B
:103220008ADB8983811509F4BECE813009F0ACC0F8
:10323000A50194012E5F3F4F4F4F5F4F2D833E837B
:103240004F835887C301B20176DB182F8A8381151B
:1032500009F4A9CE8FEF810F833058F56D817E81FF
:103260008F81988568DB8B83811511F0C601EED8BC
:103270002401350133E0430E511C611C711C47C011
:10328000B7E28B16B1E09B06A104B10409F48BCE22
:10329000C501B40150DBEFEF8E1A9E0AAE0ABE0ADA
:1032A0008111EECF0150A7CF4D805E806F80788472
:1032B0002EC08BEF810F833098F52401350143E058
:1032C000440E511C611C711C6D817E818F8198851B
:1032D00032DB8B838115D9F0C301B2012CDB8C83E7
:1032E000811571F08B819C8181305FEF950710F023
:1032F000982F8827163071F0173079F00E94D82760
:103300002401350134E0430E511C611C711C530132
:10331000420178CF0E948527F3CF0E94A627F0CFE5
:10332000143009F0C1CF6D817E818F81988503DBD8
:10333000182F2401350184E0480E511C611C711CBA
:10334000C501B4016D5F7F4F8F4F9F4FF4DA1115A8
:1033500009F429CE811509F426CE8150990B4FEF3F
:10336000489F9001499F300D1124A12FA150BB0B04
:103370002A0F3B1F2150310950F2EFE9FFE031974E
:10338000F1F700C00000F6CFC60160D8C0CF01152C
:1033900027E5120708F4A5C0011538E5130708F062
:1033A000E2C7680147E5D41A6DE773E08C2D87DC2E
:1033B000892B31F5C601E4E0880F991FEA95E1F702
:1033C000FC01E05FFB4F2281213009F05AC02091BF
:1033D0007D0330917E03232B99F020917F03309160
:1033E0008003232B69F02091810330918203409167
:1033F000830350918403242B352B232B09F44BC0DA
:1034000080918703811509F4EEC0C0909804D09094
:1034100097040E940E0888579C4E909389038093CE
:103420008803F7018581811509F4DDC08D2D8C2974
:103430008D7981110BC10115F0E51F0708F0A5C0BA
:10344000011520E4120708F008C1063E110509F431
:10345000CAC0C80190528115904208F005C1D70139
:1034600016968C91803108F4E9C0C8019927109212
:103470009A048D32910509F0A1C082E080939A04EC
:10348000F7C0223009F0BCCF209181033091820334
:10349000232B09F4B5CFFC01EB5EFB4F20812E7F7F
:1034A0002083805F9B4F0E944610AACF03375CE7C2
:1034B0001507B9F480918703811519F00E94211036
:1034C00072CD109298040E940A040E940E08885738
:1034D0009C4E909389038093880381E080938703B7
:1034E00062CD023A82E51807A9F158F4C80190525A
:1034F0008115904208F1013E110561F1053E11056B
:1035000003C0023BB2E51B0709F07ACF25EE30E09D
:103510002770332781E090E001C0880F2A95EAF7F1
:1035200020918A03309187033115E1F04115A9F00C
:10353000282B20938A0337CDF7018681803108F04C
:103540005FCF812F99278F7199278230910511F0D4
:103550004297DACF21EE30E0DBCF80958223809353
:103560008A0321CD322F3823311509F449CF982F02
:103570009095922390938A030E940204D701159696
:103580008C91811509F40FCD3BCF003EB2E51B07AE
:1035900008F047C0003CE2E51E0728F5003AF2E5D6
:1035A0001F07E8F4003622E51207E8F4C801925537
:1035B00080349105C0F010929A04C8018E329105B2
:1035C00008F063C08832910508F050C08E31910533
:1035D00008F04EC004974A9708F44FCF37C0043B19
:1035E00032E5130741F7F7013580311409F457C06C
:1035F0000E35FCE71F0709F44EC00F352CE7120704
:1036000051F00D353CE7130709F049C080912901BD
:10361000811509F440C01092290180E00E946B10CE
:10362000C2CC09374CE7140728F407375CE71507C5
:10363000D0F6C1CF0B378CE71807D4CF812F8F710D
:10364000843189F2863111F410929A040E9421107B
:1036500080918A030E94FC03C6CFD70116968C91F5
:10366000803108F002CFBFCFC80101CF8A9771F730
:1036700080918A03811531F080919A0492E0892724
:1036800080939A040E94100CAECF8C34910581F384
:103690008D329240ECCF81E08093290184CC8091DF
:1036A0002901811169C0C80197558115914008F021
:1036B000FDC05801F8EFAF22BB24A114B10409F0FA
:1036C00072CCF801FF2754E0EE0FFF1F5A95E1F787
:1036D0009F01205F3B4F6901D70115968C91EB5EEE
:1036E000FB4F908180FB90F99083811509F4D8C13C
:1036F0000E940E089093930480939204F6018281B5
:103700008F5F828380919A0490919804892B8383A0
:103710008091970484834681578166857785C601A9
:103720000E947D07D60115968C9181FF5801B092B9
:103730009104A0929004D70115969C91911509F4DB
:1037400016C610929404980130572332310508F0C0
:103750001CC684E090E00E945834909352058093F8
:103760005105F801E150F047E232F10508F0E0C1FF
:10377000E054FB4C0C94E933380150EE651A7108A3
:103780005090990480919804582A80919704582A5F
:1037900088E06816710408F05CC098012770332730
:1037A00081E090E001C0880F2A95EAF7311409F40E
:1037B0004DC0582AD7018D919C910E94840321E02D
:1037C00030E0F90102C0EE0FFF1F8A95E2F7FA8799
:1037D000E98720910604309107043E832D834091B0
:1037E0000E0450910F045C874B876DE8C62E63E092
:1037F000D62EA12CB12C511005C0D60112968C9159
:10380000811119C0F601838190E029853A858223D0
:103810009323892B81F08085982F9770911101C097
:1038200087E038E06316710408F000C1311409F430
:103830005DC081FD5DC09FEFA91AB90AAFE0CA0E55
:10384000D11CB8E0AB16B104B1F61CC0809558226B
:10385000B1CF311038C080910E0490910F04081739
:10386000190781F410920F0410920E0410920A04AA
:1038700010920B0410920C0410920D041092090483
:10388000109208048091060490910704009709F4AF
:103890000ACFE8E06E16710408F0ECC0652D0E94B6
:1038A000BC06811103C081E00E946B10F701858185
:1038B000F801E851FC47E730F10508F03CCFEE5144
:1038C000FB4C0C94E93310930F0400930E040E94F8
:1038D000270960930A0470930B0480930C0490935F
:1038E0000D04109209041092080464CF82FFA3CF44
:1038F000D6018D909C900815190519F4311409F41E
:103900009ACFED81FE81EC15FD0509F494CFD60127
:103910001D96ED91FC91309721F08081811509F47D
:103920008ACF652DC6010E94BC06811509F483CF9C
:1039300081E00815190509F080E0482E4320811424
:10394000910441F0411006C0EB85FC858E169F0660
:1039500009F071CF80E00E946B10D0920704C092F2
:10396000060481E0809305048FE08A9DF0018B9D21
:10397000F00D1124E357FC4F858180938C03411097
:103980000EC08114910459F0808191819C012450D2
:103990003109213A310508F04FC00E94FF078FE03E
:1039A0008A9DF0018B9DF00D1124E357FC4FC680DA
:1039B000D780C6019A9581159F4110F420EED2223E
:1039C00099249394C60101978F339E4708F0912C58
:1039D0008FE08A9DD0018B9DB00D1124A357BC4F61
:1039E0001996ED91FC911A97309731F01B966D91D5
:1039F0007C9181E0099598229114A9F08FE08A9D2D
:103A0000F0018B9DF00D1124E357FC4F86819781C7
:103A10000E94E70280938B03C60148E0641671049C
:103A200070F40E944B090E94100C12C0311409F46A
:103A300002CF80FD5DCFFFCE0E94BF0FB0CF0497B5
:103A4000813A910558F46C2D8EEB91E00E94E507C8
:103A5000411409F428CE0E94100CA5CA0E94100C33
:103A60008FE39CE90197F1F700C000008C2D0E94C4
:103A7000610FEECFDC012D913C910217130741F449
:103A8000311009C01092050480E00E946B100BCE2B
:103A9000311409F408CEFC01808585FD04CEF4CFF5
:103AA000F9014485558566857785C9010E947D07A2
:103AB000D60115968C9181FF3ECEC6010E942A1038
:103AC00080919004909191040817190709F033CE62
:103AD00010929104109290042ECE06E221EE41EE57
:103AE0006AE17CE71CD95FCA07E225EE45EE6BE18F
:103AF0007CE7F8CF06E221EE40EE68E17CE7F2CF0A
:103B000007E225EE44EE69E17CE7ECCF06E221EE28
:103B100042EE6CE17CE7E6CF07E225EE46EE6DE192
:103B20007CE7E0CF08E221E045EE6EE17CE7DACF0A
:103B3000809151058160809351056091510570918C
:103B4000520584E090E00E9486340E94660C2BCAE5
:103B500080915205886080935205EFCF8091510586
:103B60008260E9CF809151058460E5CF8091510555
:103B70008860E1CF809152058160EDCF8091520540
:103B80008260E9CF809151058061D5CF8091510548
:103B90008062D1CF809151058064CDCF0E94660CA8
:103BA000809151058068C7CF809151058C60C3CF4B
:103BB000809152058360CFCF809151058E7FBBCF1E
:103BC00080915205877FC7CF809151058D7FB3CFFC
:103BD000809151058B7FAFCF80915105877FABCF0F
:103BE000809152058E7FB7CF809152058D7FB3CFE4
:103BF000809151058F7E9FCF809151058F7D9BCF06
:103C0000809151058F7B97CF0E94660C8091510562
:103C10008F7791CF80915105837F8DCF8091520511
:103C20008C7F99CF80915105992782FF939590FBC6
:103C300082F990FB83F97FCF80915205982F909560
:103C400090FB80F990FB81F986CF90915105892FE7
:103C50008F7B96FF80646FCF0E94660C9091510518
:103C6000892F97FB87F9805866CF61E08EE090E05E
:103C70000E946C3462CF60E0F9CF90915105892F9A
:103C80008F7E94FF806157CF90915105892F8E7F51
:103C900090FF816050CF90915205892F877F93FFCD
:103CA000886059CF89E26EC30737BCE71B07F9F07C
:103CB0000837ECE71E0731F19801205E32452032CB
:103CC000310528F5911123C00F7181E090E09C012E
:103CD00002C0220F331F0A95E2F78901622F83E0A9
:103CE00090E00E946C34802F0E9430035CC981E018
:103CF000911551F00E94360343E062E081E00E949A
:103D0000B80351C982E0F4CF0E944003F5CF40913F
:103D1000960480915005282F30E02095309570E072
:103D200024233723232B19F04823409396040B3781
:103D30003CE7130741F4911509F435C90E941D03AE
:103D40000E94DD0630C9003442E5140708F055C072
:103D5000003252E5150708F057C0011580E5180735
:103D600050F50115A0E41A0708F064C0911509F494
:103D700079C00A35FCE71F0709F4CDC008F0B2C0CE
:103D800001303CE7130709F4C4C003304CE71407C3
:103D900009F4B9C001151C4709F064C00E94660C03
:103DA000AFEFB4E3ECE0A150B040E040E1F700C079
:103DB00000000E948C099801305521153240B0F660
:103DC000980145E0369527954A95E1F7822F8F7047
:103DD0002091960430E041E050E0082E02C0440FEC
:103DE000551F0A94E2F724233523232B09F4BECF71
:103DF0009111A6CF109298042ECE9801205C3245E6
:103E00002032310508F0B2CF802F8F7120919604B7
:103E100030E041E050E0082E02C0440F551F0A94E4
:103E2000E2F724233523232B09F4A0CF911509F4BD
:103E3000BAC886CFF7018681803108F097CF9111FB
:103E400011C0212F2F7081E090E002C0880F991FD0
:103E50002A95E2F72091960430E082239323892B60
:103E600009F0A1C8F70187819085009709F457C030
:103E70000E9408058C01F701B580A680A2942FE06E
:103E8000A22280919B048770811501F1CB2CB11483
:103E9000F1F0812F807F803461F080E2800F8830E4
:103EA000A8F0812F807E803221F4023078F0A114B6
:103EB00069F08091520582FF09C082E00E94E1030F
:103EC00080919B048770CC24C3948111C12CE12F75
:103ED000E295EF70103C08F094C0F0E0E751FB4C25
:103EE0000C94E9330B358CE71807B9F08091520533
:103EF000002482FF0394802D0C351C4709F0B2CFBB
:103F00000E94D20BAFCF6FEF7FEF80E090E00E9476
:103F100086340E94890C81E0F3CF80E0F1CF858167
:103F2000C080D180811569F0C6010E941014182F3D
:103F3000682FC6010E944E03B601812F0E94F5131F
:103F400097CFC6010E948403182FF6CFF12FFF7080
:103F5000DF2E103118F0D29490EFD922B114A9F0CD
:103F6000D11459F080E2800F883010F0011107C0A1
:103F70008D2D0E94FC030E94100C802F40C0809168
:103F80009A048D2980939A04F6CF802F0E94BF0F48
:103F9000D114B9F180E2800F883010F0011104C013
:103FA0008D2D0E94020406C0D09480919A048D2128
:103FB00080939A040E94100C24C0212F2F70D22EBF
:103FC000107F103219F0D29480EFD822011549F0F9
:103FD000013009F483C0B11409F48FC0A114A9F110
:103FE000CCCF8091520582FD2CC0B11421F1D114A7
:103FF00029F08D2D0E94FC030E94100C80E00E948D
:10400000610FC11409F4D9C080919B0480FDD5C013
:10401000D70115961C928695869586950E94360343
:10402000C7010E94EF1680919B0486958695869520
:104030000E944003C2C080E00E94BF0FD11409F368
:10404000AFCFB11469F1A11004C08D2D0E940210F0
:10405000D8CF31E0A31210C0109197048D2D812389
:10406000D81679F20E940E0890939F0480939E04C4
:104070001D2910939704C5CF45E0A412C2CF8D2D02
:104080000E9402108D2D0E942E08809199049D2D72
:104090009823D91609F4B5CF8D2980939904B1CF0F
:1040A000A11012C08D2D0E9408108D2D0E942E0887
:1040B000809199049D2D9823911509F4A2CFD09455
:1040C000D822D09299049DCF51E0A5129ACF809129
:1040D00098048D21811509F494CFE4CFB11429F00F
:1040E00086E0A81608F08DCFB0CF95E0A91608F0AD
:1040F00088CF8D2D0E94081084CFA114D1F30933ED
:1041000049F4AFEFB7EEE3E0A150B040E040E1F793
:1041100000C00000802F0E94BF0F73CF812F8695B3
:1041200086958370811561F0813009F06ACFC801EE
:104130009370B11002C080E090E00E94BD0761CF93
:10414000C8019370B11002C080E090E00E94950712
:1041500058CF6B2D802F0E946C0853CF812F837016
:10416000811139C0B11027C0402F42954695477044
:10417000440F440F802F8F70042E01C0880F0A94C3
:10418000EAF7202F207104FF07C02FE030E001C0C4
:10419000220F4A95EAF7209516951695137012305E
:1041A000A9F0133089F030914F05113061F0822B66
:1041B00083230E9430030E94820760E0C7010E94AF
:1041C0003A140C94E417832B822BF3CF822B90911B
:1041D0004F058927EECFB11451F110FFECCF402FDE
:1041E000429546954770440F440F802F8F70042EE0
:1041F00001C0880F0A94EAF7202F207104FF07C03E
:104200002FE030E001C0220F4A95EAF7209516957D
:1042100016951370123089F0133069F03091500503
:10422000113041F0822B83230E943303C4CF8230AC
:10423000B0F6C1CF832B822BF7CF822B9091500504
:104240008927F2CF1F70B11439F0812F0E943603F5
:10425000802F0E940210AFCF802F0E940810812F64
:104260000E944003A8CF023F71F170F4003FC9F0F3
:10427000013F91F0B11409F465C0A11409F45FC0C5
:10428000802F0E94610F97CF033F21F1043F91F7E8
:104290008091520582FD2AC0812F8F71B11401F3E4
:1042A00016C0B11469F0F5E0AF1608F084CF1F71A5
:1042B00081E090E0012E01C0880F0A94EAF7BECF9A
:1042C00026E0A216F2CF812F8F71B110C9CF0E94C4
:1042D000360371CF80E0B11409F4A6CF1F7181E0DD
:1042E000012E01C0880F0A94EAF79ECFB114C1F0E5
:1042F00080919B048770843049F410929B04109243
:104300009D0410929C04812F8F71AACF35E063E049
:10431000A31608F050CF812F8F710E941A084BCF3F
:1043200045E0A41640F010929B0410929D04109258
:104330009C0464E0F0CF81E00E94E1033CCF812F38
:104340008F71C5CFA114F9F2093349F45FEF87EEFD
:1043500093E0515080409040E1F700C00000802F72
:104360000E94BF0F28CF0337BCE71B070BC90631DC
:10437000ECE71E0709F098CC80919504811509F4AB
:1043800091CC85E30E94FF0766CB0631FCE71F074F
:1043900009F08ACC809198048A7A91E0811101C059
:1043A00090E09093950465E3811101C069E28EEB82
:1043B00091E00E94E5074FCBA0E0B0E0E2EEF1E231
:1043C0000C94AA338091FC02803108F049C080919E
:1043D000FB02811509F444C0C091AD0289E0D82EDA
:1043E0008091AC028C17E1F1EC2EF12CDC9EE00107
:1043F0001124FE01E255FD4F84818115B1F19181B7
:104400008091F702981331C090818091F602981341
:104410002CC08581811129C0028113818091F8020D
:104420009091F902081B190B60E086EF92E00E9460
:104430003A140E94741608171907B8F48091FC0208
:104440008F7080618093FC02CC54DD4F88818F7027
:104450008061888386EF92E00E94EF160E94D70366
:10446000CDB7DEB7E7E00C94C633E7012196C770FD
:10447000B7CFAFE0B0E0EFE3F2E20C94A2338C01EF
:1044800086E0F801DE011A9601900D928A95E1F717
:10449000F801F580E48086EF882E82E0982E8091E6
:1044A000FA02811117C0E11491F0F11409F480C1EE
:1044B000C8010E946914811509F47AC189E0F801E4
:1044C000A6EFB2E001900D928A95E1F775DFFF2427
:1044D000F3946AC0A280B380D090FB028091F8026E
:1044E0009091F9023501681A790AD11409F411C1C1
:1044F000C080518060E086EF92E00E943A140E94F2
:1045000074166816790608F0B6C0E11401F38091BC
:10451000F702F8019181E090FC02F0E1EF1608F05B
:1045200064C0981320C09091F602F801808198131E
:104530001AC02091FD023091FE02878190852817D4
:10454000390789F4F1104BC08E2D8F7080618093F4
:10455000FC0286EF92E00E94EF168091FC02F801C7
:104560008683F12C21C0F1103AC040E0652D8C2DDE
:104570000E94170B40E0652D8C2D0E94170BF82E22
:104580008111EFCF8A859B850E945C14292F22958B
:104590002F70903470F49F702230A0F09115B1F01C
:1045A000F8019681903190F48F2D2F96EFE00C94C6
:1045B000BE332A5F2F70223068F0C8010E94EF16C8
:1045C000FD2CF2CF911511F0811571F3805E8830CA
:1045D00058F3F3CF803F40F3815F8330F9CF809170
:1045E000FC0281608093FC02BCCF98131EC09091A6
:1045F000F602F8018081981318C02091FD023091D5
:10460000FE02878190852817390779F4F1100DC0D3
:10461000E682C8010E94EF1689E0F801A6EFB2E039
:1046200001900D928A95E1F752CFC8010E9469145A
:10463000811509F4BDC0F11409F4BAC08091FC02DF
:10464000803208F43BCF8091F6029091F7029A8372
:104650008983BC82AB828091FA028D831E82EF82B5
:104660008091FD029091FE0299878887CE01019684
:104670000E94EF1623CFD090FC02F0E1DF1650F439
:1046800086EF92E00E94EF1689E0F40111928A957C
:10469000E9F767CFE11409F41ACF9091F702F80116
:1046A000818198131AC09091F6028081981315C0E9
:1046B0002091FD023091FE028781908528173907ED
:1046C00061F4F1100AC0D682C8010E94EF1689E099
:1046D000F40111928A95E9F7FACEC8010E94691493
:1046E000811509F465C0F11409F462C08091FC02DF
:1046F000803208F4E3CE8091F6029091F7029A831B
:104700008983BC82AB828091FA028D831E82DF8214
:10471000A7CF60E086EF92E00E943A140E947416E0
:104720006816790608F0B0CFE11409F4D0CEF11480
:1047300009F43EC09091F702F801818198132EC0D0
:104740009091F6028081981329C02091FD0230914A
:10475000FE02878190852817390701F58091F802BC
:104760009091F902A81AB90AF8ECAF16B10408F052
:1047700053CF8091FC0280FD4FCF803108F44CCFA5
:10478000F8018683982F907F903F09F442CF982FAD
:10479000907F905F8F70892B86833BCFC8010E94EA
:1047A000691481118BCE8091FC0281608093FC02A0
:1047B000C8010E94EF168BCEA2E1B0E0E2EEF3E278
:1047C0000C94AD330A871B872C873D874E875F8704
:1047D000688B798B8A8BCE010A964BDE811128C0BB
:1047E0002091AC023091AD0289E0FE013A96DE01E3
:1047F000119601900D928A95E1F78E858115C1F091
:10480000822F90E001968770992738171906D9F002
:1048100099E0929FD0011124A255BD4FFE0131961F
:1048200001900D929A95E1F78093AC020E94D70314
:1048300019E08091AD029091AC02891312C062968A
:10484000E4E00C94C9330E94660C1092AC02109202
:10485000AD0289E0E6EFF2E0DF011D928A95E9F70B
:10486000E7CF189FC001112482559D4F02DE8115AC
:1048700031F38091AD0290E0019687709927809383
:10488000AD02D7CFEF92FF920F931F93CF93DF9399
:1048900080914C05E091EE01CDE0811130C0CDB7A3
:1048A000DEB7E6E00C94C733D1E0DE0FD093EE0123
:1048B000EE2EF12CCE9FF0011124EC51FB4F8481A0
:1048C0008115E1F087819085892B21F4818592857E
:1048D000019651F4008111812281338144815581F7
:1048E00066817781808568DFCE9DF001CF9DF00DD8
:1048F0001124EC51FB4F148210929A04ED2F8091F9
:104900004C05E81788F210924C051092EE01C7CFC3
:10491000A4E0B0E0EEE8F4E20C94A0332091E304CC
:10492000298397E0992E01E010E02DE0322E34E04B
:10493000532E882483948091E2049981891307C0BF
:10494000A1DF0E947F062496E1E10C94BC3399819B
:10495000892F90E09C838B83FC01EE0FFF1FE852B0
:10496000FB4F80819181989ED001999EB00D1124BA
:10497000FD01E056FB4FFA83E983248121115BC0DE
:1049800060904C05E4EEF4E060E070E0712C661598
:1049900008F04FC0A384B484A981BA81CD90DC9083
:1049A0002FEF3FEF412C442D50E07601E40CF11C39
:1049B000E40CF11CD701ED90FC90E114F10439F006
:1049C000AE14BF0409F0A90143949A01ECCF2F3F24
:1049D0003207D1F1D80102C0AA0FBB1F2A95E2F716
:1049E0007A2A9801042C02C0220F331F0A94E2F79E
:1049F000A901415051097416150629F5369EF0019A
:104A0000379EF00D1124EC51FB4F989ED001999EDA
:104A1000B00D1124A056BB4F12962D913C911397C7
:104A2000308727835482108211829287818715965E
:104A30008C920E9490068B819C8101969A83898337
:104A40008370898378CF14826F5F7F4F3D969FCFAD
:104A500010924E0510924D0510922A018091E204A9
:104A60008093E3040E947F060DCFACE1B0E0EBE35E
:104A7000F5E20C949F334B8B5C8B6D8B7E8B8F8B15
:104A8000B92E988FA92E911110929A04188A198A1A
:104A90001A8A86E0FE017396DE011A9601900D9245
:104AA0008A95E1F75F888091520582FF1FC00E94BE
:104AB0000E0820919C0430919D04821B930B883832
:104AC000934138F080919B0482FD03C082E00E94F4
:104AD000E1030E940E0820919E0430919F04821BE6
:104AE000930B8838934110F00E940A045114D9F0B6
:104AF0005E86BF8661E0CE010A960E943A1461E0AC
:104B0000CE010A960E943A1461E0CE010A960E94F4
:104B10003A144C0180356CE7960791F4A11419F111
:104B200081E080932A015E86BF860A851B852C85DD
:104B30003D85452D5B2D688979898A893DDECDC00B
:104B400081359C4721F4A11471F082DFECCF82E51E
:104B500088168CE7980639F4A11429F080912A016F
:104B60008111F3CFDDCF40EAE42E44E0F42E412C56
:104B7000612C712CD7016D917C91CC24CA94DD24D9
:104B8000DA9480E0282F30E0FB01E80FF11DE80FF8
:104B9000F11D408151814115510539F0841695066A
:104BA00009F096018F5F6901EDCF10E0BFEFCB16E2
:104BB000DB0609F44EC0F701448110912A0141112E
:104BC00010E0D70115963C90159716969C91169774
:104BD000A11409F405C1111509F402C1311017C05F
:104BE00021E030E00C2C01C0220F0A94EAF7922B4E
:104BF00016969C932091E0043091E1042233310514
:104C000030F422E330E03093E1042093E004E1E06B
:104C1000F0E002C0EE0FFF1F8A95E2F7CF01019787
:104C2000D70116962C912817190699F4C0904D05B6
:104C3000D0904E05C114D10409F453C00E940E084F
:104C40008C199D09C39708F44CC081E0F701848357
:104C500011E0412ABFEF6B1A7B0AE7E0EE0EF11C70
:104C6000F8E06F16710409F085CFA11409F417C19B
:104C7000411409F414C10E940E0890934E058093CC
:104C80004D0580914C05883040F591E0980F909348
:104C90004C0599E0FE013A96DE01119601900D92C5
:104CA0009A95E1F75D82BE822DE0829FC0011124BA
:104CB0008C519B4F29E0FE013196DC0101900D9251
:104CC0002A95E1F72FEF3FEFDC011A963C932E93E4
:104CD00019971C969C928E921B976C96E2E10C940D
:104CE000BB332091E3048091E204922FE0E0F0E0F6
:104CF00001E0281709F448C0422F50E0FA01EE0FF6
:104D0000FF1FE852FB4F2080318037E0329DF001D9
:104D1000339DF00D1124E056FB4F608171817C8F33
:104D20006B8FB0E030E0A0E0EB8DFC8DEA0FF11D61
:104D3000EA0FF11DC080D180C114D104E1F0F70168
:104D40000190F081E02DFA8FE98F30E007C0E1E0BB
:104D5000C616D70609F0E0E0BE2B3F5FE98DFA8D5D
:104D6000E30FF11DE30FF11D608171816115710584
:104D700071F7AF5FD9CFB11581F13A17C8F4E1E00F
:104D8000D7011496EC93F7019093E304EE15FF0519
:104D900009F45FCF90E0FC01EE0FFF1FE852FB4FDC
:104DA000718260820196837099278093E20451CFCB
:104DB00037E0329DF001339DF00D1124E056FB4F9A
:104DC0000483EE15FF05F9F2291302C09F5F93706B
:104DD0009A012F5F3F4F23708CCFE0E0F0E0F8CFD7
:104DE000292F30E0311024C061E070E002C0660F6E
:104DF000771F8A95E2F7CB0101972817390791F0C1
:104E000010E0E1E0F0E002C0EE0FFF1FCA94E2F70D
:104E10006F01C094D70116968C9116978C21169627
:104E20008C9317CF411569F3C3010E949006E8CF18
:104E3000A9010C2C02C0559547950A94E2F7C901C7
:104E4000019782239323892B39F540FF25C0D70191
:104E500012968D919C91892BD1F087E0FE013196BD
:104E6000DF011D928A95E9F70E940E089C018B8351
:104E70009C8384E08D83F70192818381792F9887C9
:104E8000898709811A8144E05E816F8195DCD701B1
:104E900015961C92132DB5CF142F1170B2CF90918F
:104EA000E3048091E204981731F032DDB1E04B1653
:104EB00009F413CF38CEE6DC10924E0510924D0562
:104EC0000E947F06F3CFA6E0B0E0E9E6F7E20C949B
:104ED000AD330E940E088C018091A0029091A10236
:104EE0008017910771F019821A820E940E08BC0186
:104EF00049815A8180E090E0B8DD1093A1020093CF
:104F0000A0022696E4E00C94C933A6E0B0E0EBE8FA
:104F1000F7E20C94AF3390939D0280939C0281152D
:104F200020E2920730F40E94AA0F2696E2E00C9449
:104F3000CB3380EF89838A830E940E088160BC0195
:104F400049815A8181E091E090DDEFCFA6E0B0E0A9
:104F5000ECEAF7E20C94AD338C0190939D028093C0
:104F60009C02011580E21807B0F4802F0E94BF0F49
:104F7000C801805E9109089728F067E170E101158A
:104F8000110511F468E070E1C8010E941103269632
:104F9000E4E00C94C93380EF89838A830E940E0871
:104FA0008160BC0149815A8181E090E05EDDEFCFF4
:104FB000CF93DF93D82FC92FA8DF8D2F9C2FC6DF6B
:104FC000DF91CF9108950F931F93CF93DF938C01BF
:104FD000862F6DE773E00E945F16892B91F4C091D4
:104FE0007D03D0917E03209761F0F80182818330A8
:104FF00039F4CE01DDDFCE01DBDFCE01D9DF01C028
:10500000E0F7DF91CF911F910F9108950F931F93B8
:10501000CF93DF938C01EB016DE773E08C2F0E943F
:105020005F16892B09F057C0FE01FF27D8011296A1
:105030008C911297E05CFD4F8130A9F415968C910C
:1050400082FD4EC080FF4CC082E0808380917F0350
:10505000909180030097B9F480917D0390917E0335
:105060000097C9F110C08230A1F515968C9182FD90
:1050700026C080FD0AC083E08083809181039091E7
:1050800082030097F1F041DF26C084E080838091A5
:105090008303909184030097B1F780917D039091F1
:1050A0007E03009701F184DF80917F03909180035C
:1050B000009749F780917D0390917E03E4CF85E0CE
:1050C000808380917D0390917E03009721F070DFB3
:1050D000F1CF86E08083DF91CF911F910F910895EA
:1050E00081E08083B9CF80917F0390918003B8CF16
:1050F0000F931F93CF93DF938C01EB016DE773E068
:105100008C2F0E945F16892B71F4DD27C05CDD4F68
:105110008881F801128218828330E9F048F48130E6
:1051200059F0823081F0DF91CF911F910F91089556
:105130008430B1F08530B9F780917D0390917E0382
:10514000009789F306C080917F03909180030097B8
:1051500099F3FCDEE8CF8091810390918203F7CF31
:105160008091830390918403009799F720917D03A8
:1051700030917E0380917F0390918003211531054A
:10518000F9F2009731F7C901E4CFA0E1B0E0EBEC10
:10519000F8E20C94A133FE01319680E1DF011D920B
:1051A0008A95E9F703E110E099EDA92E92E0B92E76
:1051B00027E2422E55245394612C712C4F01730128
:1051C0006201B1E14B165104610471041CF080E1ED
:1051D000C82ED12CA601B501C4010E945D34AC0CCF
:1051E000BD1C0D2C000CEE08FF084C185D086E0865
:1051F0007F080150104019F76096E0E10C94BD3330
:105200006FEF85E290E00E946C346FEF86E290E0F1
:105210000E946C346FEF87E290E00E946C3460E093
:1052200088E290E00E946C340E94C514AEDF62EA0E
:1052300085E290E00E946C346DEA86E290E00E9484
:105240006C346BE687E290E00C946C34CDB7DEB73B
:10525000AC970FB6F894DEBF0FBECDBF85B78068A0
:1052600085BF85B7806885BF84B7877F84BF0FB649
:10527000F894A895809160008861809360001092F6
:1052800060000FBE80E890E00FB6F8948093610054
:10529000909361000FBE81E08093030184E096E06B
:1052A0009093BD018093BC010E942C060E945C1566
:1052B0000E94A0150E941F160E94470A0E94BD0A64
:1052C0008091E20084608093E200789480917E0275
:1052D000811599F08091E9001091EC008F7017957D
:1052E00011271795182B1092E9008091E80083FD93
:1052F0000E949E0C1F701093E90082E084BD93E031
:1053000095BD9AEF97BD80936E001092980210920F
:10531000990210929A0210929B020E94AC14811181
:1053200001C06EDF8091D80080618093D8002AE1AF
:105330002A95F1F700C08091D900182F117080FDD7
:1053400004C00E94470A10927E02109396021093A6
:1053500097021093040111110E944C3280910401B4
:105360008091040190E0811101C095E09093530277
:1053700085E0891B8093520203E411E0D8018D91EE
:105380008D018F3F11F00E940606B1E008341B0723
:10539000A9F708E411E0F80181918F018F3F11F026
:1053A0000E940606F1E00D341F07A9F78AE0E2E744
:1053B000F2E0DF01282F1D922A95E9F7E8E4F2E0F8
:1053C000DF011D928A95E9F780E090E00E94583451
:1053D000833E9E4F21F40E94AC14811128C063EEDD
:1053E0007EEF80E090E00E94863460E082E090E012
:1053F0000E946C3481E080934F0561E083E090E08F
:105400000E946C3460E074E184E090E00E94863495
:10541000F7DE40E050E0BA018FE090E00E947E3479
:1054200040E050E0BA0183E190E00E947E3482E0E7
:1054300090E00E9450348093560284E090E00E94F5
:10544000583490935205809351050E94C610EFEF97
:10545000F6E721E0E150F0402040E1F700C0000015
:105460000E94C6108091720280FF08C06FEF7FEF2C
:1054700080E090E00E9486340E948C0983E090E0F6
:105480000E9450340E94300380919602811102C024
:105490000E944F3285E091E09093A3028093A20294
:1054A00080917E02853049F480917E02853009F436
:1054B00050C00E94660C0E9482070E94C61007E539
:1054C00012E052E7E52E52E0F52ED701F801919156
:1054D0008D9121E632E02E173F0709F46FC098172F
:1054E000B1F380909602D12CD701CD907D01F801C7
:1054F00091908F019C1431F19C24B12CAA24A39487
:10550000892D8A218115B9F08114A9F0B982DA8236
:105510000E940E089C838B83F1E0FD8391E08C2D2B
:105520008A21811101C090E09E8349815A816B815B
:105530007C818D819ADAB394AA0C25E0B212E0CF77
:10554000F801C292D3943AE0D312CECF0E9433092D
:1055500038C080917E02843021F11092540288E19B
:1055600090E0A0E40FB6F894A895809360000FBE79
:10557000A093600083B7817F846083BF83B781601D
:1055800083BF7894889583B78E7F83BF0FB6F894D6
:10559000A8958091600088618093600010926000FF
:1055A0000FBE0E94C610E2E7F2E08191811186C52C
:1055B0002CE732E02E173F07C1F776CF981391CF33
:1055C00082DC80919602811509F49EC00091080446
:1055D000109109040115110591F1C0906502D09058
:1055E0006602E0906702F09068020E9427096C1939
:1055F0007D098E099F09C0906102D0906202E090FF
:105600006302F09064026C157D058E059F05B8F06D
:10561000C8010E94AA0F1092090410920804109267
:105620006502109266021092670210926802109250
:105630006102109262021092630210926402E09082
:105640009004F0909104E114F10439F1C0909204B7
:10565000D09093040E940E088C010C191D09C701FB
:105660000E94741680179107C0F420919004309125
:105670009104C9019927287F3327232B09F05BC1A7
:1056800044E0880F991F4A95E1F7805F9B4FDC014A
:1056900015962C9122FF0E94461080912A018115B7
:1056A00011F100914D0510914E0501151105D9F02C
:1056B0000E940E08801B910B2091E0043091E104C0
:1056C0002817390780F49091E3048091E204981739
:1056D00009F434C11DD91092E1041092E004109233
:1056E0004E0510924D0580918703811569F00E9447
:1056F0000E082091880330918903821B930B8F3F02
:105700009F4710F40E94211086E0E7E1F3E0DE01FC
:10571000119601900D928A95E1F7B0901803D09000
:10572000190310911A03C0901B0300911C031092DF
:10573000190310921A0310921B0310921C03812F5D
:105740008D29811509F441C0E0906B02F0906C0244
:105750000E940E089C012E193F0990911503911586
:1057600009F4A7C42531310580F19F3F19F09F5FEF
:1057700090931503D11459F00E94120791E01D1463
:105780000CF09FEF899F802D112480931903111530
:1057900059F00E94120791E011160CF09FEF899FBB
:1057A000802D112480931A0380911903811569F0CB
:1057B000F0901A03F11449F00E9404078093190332
:1057C0008F2D0E94040780931A038C2D802B811546
:1057D00009F441C0E0906902F0906A020E940E084C
:1057E0009C012E193F0990911403911509F45CC492
:1057F0002135310580F19F3F19F09F5F909314038D
:10580000C11459F00E94320791E01C140CF09FEF74
:10581000899F802D112480931B03011559F00E944C
:10582000320791E010160CF09FEF899F802D112414
:1058300080931C0380911B03811569F0F0901C0379
:10584000F11449F00E94040780931B038F2D0E94DE
:10585000040780931C03809118038B1119C0809159
:105860001903811511F08D1113C020911A03211510
:1058700011F021130DC090911C03911511F090139C
:1058800007C030911B03311103C0822B892B81117A
:105890000E94430886E0FE013196A7E1B3E0019043
:1058A0000D928A95E1F70E94820790916D02891707
:1058B00021F080936D020E94270980917E0284303E
:1058C00009F0EECD83E08093E9008091E80082FF4B
:1058D000E7CD8091E80090E085FF0BC00E94160A9A
:1058E00030E2E32EF12C8E010F5F1F4F8115C1F1C5
:1058F00091E08091E8008B778093E800911509F49E
:10590000CFCD00919E0210919F02E98101151105F2
:10591000A9F1EE3F09F054C08A81833020F0855010
:10592000833008F04DC0EA81EE3008F049C0F0E065
:10593000EB50FB4C4EC780E090E0A9CE0E94422481
:1059400010924E0510924D050E947F06CCCE80919C
:10595000F100F80181938F01F1E0EF1AF10841F2B3
:105960008091E80085FDF3CF8091E8008B778093EC
:10597000E8000E94160A811599F3BACFE43148F481
:10598000E11549F0E150E33130F4F0E0ED5FFA4C1D
:1059900020C7EE3F41F28FEF898312C01A8289E05F
:1059A0008B830EC08A81823081F08330B1F08130E8
:1059B00091F70E94270923D76B837C838D839E8375
:1059C000CE0101960E94660A6BCD88E290E068D70E
:1059D0001B821C821D828E83F3CF80917C0290916A
:1059E0007D02892B69F38AE0E2E7F2E0DE0113969B
:1059F00001900D928A95E1F7E3CF8A81823059F6C2
:105A00006B817C818D819E81FAD688E290E064D79B
:105A1000D7CF4C816B818A810E94C6139827892732
:105A200098279E838D83CCCF2D813E8132272327DB
:105A300032274C816B818A810E94E90BC1CF0E9481
:105A4000C514BECF80E18A83BBCF81E08A8387E221
:105A5000A7CF8C818D3108F0B3CF8A809B809824AA
:105A600089249824A12CB12C9E012F5F3F4F7901EE
:105A70008901080F111DE016F10609F4A1CF80E09D
:105A800037E2831631E09306A104B10420F4C40187
:105A900087529D4F05D7D70114968C93BFEFEB1A11
:105AA000FB0AEFEF8E1A9E0AAE0ABE0AE4CF80917F
:105AB0007C0290917D02892B09F482CF8C818D31FB
:105AC00008F07ECF882E912CA12CB12CCA80DB80CF
:105AD000DC24CD24DC24E12CF12C8E010F5F1F4F40
:105AE000412C512C3201481459046A047B0408F0FB
:105AF00067CFF7E2CF16F1E0DF06E104F10438F4F6
:105B0000D80114966C91C60187529D4FE5D6BFEF20
:105B10004B1A5B0A6B0A7B0AEFEFCE1ADE0AEE0A1B
:105B2000FE0A0F5F1F4FDFCF30DB4ACF84E08BCF01
:105B30008C818D3108F044CF882E912CA12CB12C72
:105B4000CA80DB80DC24CD24DC24E12CF12C412C28
:105B5000512C32018E010B5F1F4F481459046A0407
:105B60007B0408F02DCF80E0F0E9CF16F1E0DF06EE
:105B7000E104F10418F4C601899692D6D8018D93F8
:105B80008D01BFEF4B1A5B0A6B0A7B0AEFEFCE1A4F
:105B9000DE0AEE0AFE0AE1CF2C81022F10E02D3141
:105BA00008F00ECF8A819B819827892798272C019E
:105BB000612C712C8039F1E09F0708F001CF822E13
:105BC000912CA12CB12C40E951E060E070E0441927
:105BD000550966097709421751056105710508F4F1
:105BE000EFCE20917C0230917D02232B09F03EC044
:105BF0001C0129E2220E311C80FBEE24FF24E0F878
:105C000080FF0BC088964CD69D81892798278927CD
:105C100081159C4711F48FEF8D83D501C401840D4C
:105C2000951DA61DB71D80FF19C0680181E0C81A27
:105C3000D108DE011596AC0DBD1DBCA7ABA7C101F7
:105C4000800F911F2DD6EBA5FCA5908181159C4757
:105C500021F48FEFABA5BCA58C938601FE01319694
:105C6000EE0DFF1D2FEFE016F10638F08E010F5FED
:105C70001F4FC12CD12C760125C0948185818115BF
:105C80009C4711F42483258332E0E30EF11C329605
:105C9000EACF80E9481681E058066104710430F4C7
:105CA000D80114966C91C201899616D6BFEFCB1A13
:105CB000DB0AEB0AFB0AEFEF4E1A5E0A6E0A7E0A57
:105CC0000F5F1F4FC814D904EA04FB0410F378CE09
:105CD00080917C0290917D02892B09F471CECE01D6
:105CE00001960E94660AFFEF21EE34E0F150204059
:105CF0003040E1F700C00000BFCB88E0EBE2F1E00C
:105D0000DE01919601900D928A95E1F7FE0132969F
:105D10008FE1DF011D928A95E9F786E0898388E0AB
:105D20007F96DE01159664CE80EE89831A821B82EF
:105D30001C8246CE8B819C81092E000CAA0BBB0BCA
:105D400025E0880F991FAA1FBB1F2A95D1F7AC0128
:105D5000BD01405E5F4F6F4F7F4F481759076A077D
:105D60007B0708F42DCE803E9105A105B10508F012
:105D700027CE413E51056105710520F040EE50E00F
:105D800060E070E0481B590BBC016E577B4FCE01A1
:105D9000019650D515CE4AE150E06FEF70E0CE018C
:105DA000079667D580917C0289830A831B821C82B7
:105DB0001D8281E010CE81E090E090939F0280935D
:105DC0009E0282E390E090937102809370020E94A1
:105DD0000E0890936F0280936E02F2CD01151105AB
:105DE00071F1D0907202E0906E02F0906F020E940A
:105DF0000E088E199F098536910540F1D1FE26C007
:105E0000D0FE24C00E940E0890936F0280936E0211
:105E1000809170029091710201979093710280932A
:105E20007002892B61F410929F0210929E0281E011
:105E300090E090937D0280937C0200E010E08091DE
:105E40007C0289830A8380917002AACD82E390E06C
:105E50009093710280937002F2CF10927D021092A3
:105E60007C02AECD40E250E06FEF70E0CE010196D3
:105E700000D5A6CDEB81E93008F0A2CDF0E0EA5ED6
:105E8000FA4CA7C4FE0135968BE1DF011D928A957D
:105E9000E9F788E089838A838B838C8383E088A3F6
:105EA0008FCD8C819AE0F92E8E010F5D1F4FF80186
:105EB0002F2D11922A95E9F7B8010E945F16898368
:105EC000F801DE01129601900D92FA94E1F778CD77
:105ED0001C818AE0FE013596DE01919601900D92BB
:105EE0008A95E1F789A19AA10E941F069AA389A326
:105EF0008BA19CA10E941F069CA38BA38DA19EA198
:105F00000E941F069EA38DA38FA198A50E941F0625
:105F100098A78FA38FEF183060F43AE0139FB00179
:105F2000112467547E4F4AE050E0CE018196F2D4AE
:105F300080E089830E942C0643CD2C816AE0CE014B
:105F40008196DC01E62F1D92EA95E9F7283008F0EA
:105F500044C0629FB0011124675F7D4F4AE050E06A
:105F60008FD480E089838AE0FE01B196DE0112962B
:105F70003FCD1C818AE0FE013596DE0191960190AD
:105F80000D928A95E1F789A59AA50E941F069AA706
:105F900089A78FEF183060F4FAE01F9FB001112439
:105FA000675F7D4F4AE050E0CE018196B3D480E038
:105FB00089830E945C1504CD2C816AE0CE01819614
:105FC000DC01E62F1D92EA95E9F7283030F4629F54
:105FD000B0011124675A7D4FC1CF8FEFC3CF1C8111
:105FE0008AE0FE013596DE01919601900D928A9528
:105FF000E1F78BA19CA10E941F069CA38BA38FEFAE
:10600000183060F4FAE01F9FB0011124675A7D4FE9
:106010004AE050E0CE0181967DD480E089830E94E1
:10602000A015CECC2C8166E0CE018196DC01E62F56
:106030001D92EA95E9F7283060F4629FB0011124BF
:1060400067557D4F46E050E01BD480E0898386E0B1
:106050008BCF8FEFFBCF1C8186E0FE013596DE01F2
:10606000919601900D928A95E1F789A19AA10E94DB
:106070001F069AA389A38BA19CA10E941F069CA323
:106080008BA38FEF183060F4F6E01F9FB00111244E
:1060900067557D4F46E050E0CE0181963BD480E0CD
:1060A00089830E941F168CCC2B30310508F0A5CBBC
:1060B000D2CB2B30310508F05ACB87CB80915502DB
:1060C000811509F4F1C930E139BD82E189BD09B416
:1060D00000FEFDCF8091D8008F7D8093D800809105
:1060E000E00082608093E0008091E00081FDFCCFC1
:1060F0000E94660CD9C91F921FB61F9211248F935C
:106100009F93AF93BF9380915402811113C08091EC
:10611000E6019091E701A091E801B091E901419673
:10612000A11DB11D8093E6019093E701A093E801C2
:10613000B093E901BF91AF919F918F911F901FBEC6
:106140001F90189578941F921FB61F9211248F9359
:106150009F93AF93BF938091E6019091E701A09147
:10616000E801B091E9010196A11DB11D8093E601FE
:106170009093E701A093E801B093E901BF91AF913B
:106180009F918F911F901FBE1F9018951F920F9285
:106190000FB60F9211242F933F934F935F936F93FA
:1061A0007F938F939F93AF93BF93EF93FF938091D0
:1061B000E10082FF09C08091E20082FF05C080916A
:1061C000E1008B7F8093E1008091DA0080FF24C0A2
:1061D0008091D80080FF20C08091DA008E7F80936C
:1061E000DA008091D90080FFA9C080E189BD82E1F9
:1061F00089BD09B400FEFDCF81E080937E028091CD
:10620000D501811109C00E94470A0E94BD0A8091F0
:10621000E20084608093E2008091E10080FF1AC078
:106220008091E20080FF16C08091E2008E7F809313
:10623000E2008091E20080618093E2008091D800CA
:1062400080628093D80019BC85E080937E0283E051
:10625000809303018091E10084FF2FC08091E200D0
:1062600084FF2BC080E189BD82E189BD09B400FEB5
:10627000FDCF8091D8008F7D8093D8008091E10080
:106280008F7E8093E1008091E2008F7E8093E20018
:106290008091E20081608093E2008091D4018115B9
:1062A00009F452C084E080937E0280917E028430A3
:1062B00009F052C082E0809303018091E10083FFE6
:1062C0002CC08091E20083FF28C08091E100877F8D
:1062D0008093E10082E080937E021092D40180914D
:1062E000E1008E7F8093E1008091E2008E7F8093B9
:1062F000E2008091E20080618093E20042E060E091
:1063000080E00E948D0A8091F00088608093F00008
:1063100081E08093030180930201FF91EF91BF918F
:10632000AF919F918F917F916F915F914F913F912D
:106330002F910F900FBE0F901F90189519BC1092BF
:106340007E021092D50168CF8091E30087FF02C0E2
:1063500083E0A9CF81E0A7CF81E0ADCF1F920F925C
:106360000FB60F921124EF92FF920F931F932F936A
:106370003F934F935F936F937F938F939F93AF93CD
:10638000BF93CF93EF93FF9309EE10E0F801808164
:10639000C091EC008F70C795CC27C795C82B108291
:1063A00080EFE82EF12CF7018081877F808378943D
:1063B0000E949E0CF8011082F70180818860808322
:1063C000CF70F801C083FF91EF91CF91BF91AF9152
:1063D0009F918F917F916F915F914F913F912F91FD
:1063E0001F910F91FF90EF900F900FBE0F901F9095
:1063F00018958EE1489B02C08A95E1F7489BFECF35
:106400000895589880E28A95F1F7589A0895FC010A
:106410002BE02A95F1F728E090E080E031E040E1C0
:106420004A95F1F7880F489B02C08160932742E0AC
:106430004A95F1F7000040E14A95F1F72A9579F77E
:1064400020E12A95F1F729B132E03A95F1F7000001
:1064500040E14A95F1F7217092272081920F9083B5
:106460000895A1E0B0E0E6E3F2E375C119828C0182
:106470007C01E60EF11CBDDFCE010196C8DFF801FC
:1064800081938F01EE15FF05B1F781E0998191119C
:1064900080E02196E6E07BC1509A589A0895509882
:1064A000589AE89AE9E6F0E080818C7F808308952D
:1064B0006150770B91E001C0990F6A95EAF7692F57
:1064C00090E021E0611108C0911599F0589A80E29E
:1064D0008A95F1F758980895362F3823311539F0F9
:1064E000589A922730E23A95F1F76695EBCF589893
:1064F000F9CF5898ECCFFF920F931F93CF93DF9370
:10650000EC018C01060F111DF9907BDF68E08F2DE7
:10651000CFDFC017D107C1F7CDB7DEB7E5E038C18F
:106520001F920F920FB60F9211240F931F932F9368
:106530003F934F935F936F937F938F939F93AF930B
:10654000BF93EF93FF93CF93DF930F92CDB7DEB757
:1065500019824FDFCE0101965ADF082F0695069566
:106560000695982F92959570202F2570920F292FC0
:10657000237096959695920F982797708981892B0D
:10658000811509F058C0043008F055C080E18A95A3
:10659000F1F7589A509A82E08A95F1F700C058981E
:1065A00088E0089F80011124D801AF5EBE4F169687
:1065B000ED91FC9117973097A9F060914D01709182
:1065C0004E0114962D913C911597260F371F119669
:1065D0008D919C911297680F791F13964C91139788
:1065E0008C910995F801EF5EFE4F6381611549F0CA
:1065F00020914D0130914E0184819581820F931F2E
:106600007ADFFFDE80E18A95F1F758985098589A22
:1066100080E18A95F1F7F801EF5EFE4F6081611528
:1066200049F020914D0130914E0181819281820F7C
:10663000931F17DFDEDE0F90DF91CF91FF91EF9177
:10664000BF91AF919F918F917F916F915F914F918A
:106650003F912F911F910F910F900FBE0F901F90A0
:1066600018950F931F93CF93DF938C0104970CF031
:106670005EC0F894509A589885E08A95F1F700002A
:10668000C02FC695C570802F8570C80F8C2F837062
:10669000C695C69593E0000F111F9A95E1F7C80FB4
:1066A000C8018C2BEC01ADDE00C068E08C2F00DF50
:1066B00090E19A95F1F75098589A489B31C087E03D
:1066C00090E048992FC0F801EF5EFE4F638161159D
:1066D00059F020914D0130914E0184819581820FB6
:1066E000931FBFDE811501F184DE80E28A95F1F708
:1066F0005898509A90E19A95F1F7F801EF5EFE4FA5
:106700006081611549F020914D0130914E018181E8
:106710009281820F931FEFDE74DE789481E008C0CF
:1067200000C0CBCF019749F4509A589A789480E0F2
:10673000DF91CF911F910F91089500C0C2CF2F928A
:106740003F924F925F926F927F928F929F92AF9201
:10675000BF92CF92DF92EF92FF920F931F93CF934E
:10676000DF93CDB7DEB7CA1BDB0B0FB6F894DEBFE5
:106770000FBECDBF09942A88398848885F846E840B
:106780007D848C849B84AA84B984C884DF80EE8055
:10679000FD800C811B81AA81B981CE0FD11D0FB65E
:1067A000F894DEBF0FBECDBFED01089597FB072E15
:1067B00016F4009406D077FD08D028D007FC05D049
:1067C0003EF4909581959F4F0895709561957F4F08
:1067D0000895EE0FFF1F0590F491E02D0994082E07
:1067E000817006940694811D0694811D0694811D76
:1067F0000694811D0694811D0694801D08956927C5
:10680000962769277827872778270895AA1BBB1B17
:1068100051E107C0AA1FBB1FA617B70710F0A61BA0
:10682000B70B881F991F5A95A9F780959095BC01C1
:10683000CD010895FB01DC0102C005900D9241508D
:106840005040D8F70895FB01DC0104C08D91019000
:10685000801921F441505040C8F7881B990B0895C6
:10686000FB01DC0102C001900D9241505040D8F76D
:106870000895DC0101C06D9341505040E0F7089548
:10688000DC01CB01FC01F999FECF06C0F2BDE1BDF0
:10689000F89A319600B40D9241505040B8F70895DF
:1068A000F999FECF92BD81BDF89A992780B50895D8
:1068B000A8E1B0E042E050E0E5CFDC01A40FB51F55
:1068C0004150504040F0CB01840F951F2E9105D0D0
:1068D00041505040D8F70895262FF999FECF92BD28
:1068E00081BDF89A019700B4021639F01FBA20BD95
:1068F0000FB6F894FA9AF99A0FBE08950396272FC7
:10690000ECDFEADF252FE9DF242FE7CF0196272FE1
:10691000E4DFE2CFDC01CB0102C02D9105D0415074
:106920005040D8F70895262FF999FECF1FBA92BD8F
:1069300081BD20BD0FB6F894FA9AF99A0FBE019660
:106940000895F894FFCF78087D087F08840894089C
:106950009408940894089408940894089408860865
:106960008A088D089208A208A808AC087B0DA10D22
:10697000A70DA10DA70DF90D1A0EA70D200F2D0FB4
:10698000DC1D441EE41DAE1DB21DE81DB61DEC1D30
:10699000F81DC21D3D1EC61DFC1DCA1D001E251E64
:1069A000CE1D041E2C1ED41D0A1E121EBA1DF01D63
:1069B000BE1DF41DD81D0E1E1C1E351E3B1EA81D1F
:1069C000E01D4B1E7A1D801D6D1D741D861D8C1DC6
:1069D000921DA61FA61FDD1FDD1F8E20A9200120EE
:1069E0000120AE202221332133217D2E942E9A2E98
:1069F000E02CE02CCB2EDB2EEE2E2D2F322FE02C98
:106A0000E02CE02C3A2FCE2CD22CFD2C092D142D6D
:106A10001F2DCB2CCB2CCB2CCB2C682E222D252D17
:106A2000292D572D942D962D982DCC2D422F512F59
:0E6A3000682F9D2FB92FDC2FEF2F12302B3047
:106A3E0000000100010B08780B9D098E0B930B6F64
:106A4E000B00000001000000000000000501000026
:106A5E00000406000000000000010189FBBB3CA4FD
:106A6E007546110044227B49012701AC004F026894
:106A7E00028802F6F73133329497C634358302E238
:106A8E0000E900EA00B500B600B700CD008301CCE6
:106A9E00008A01920194012102230224022502267A
:106AAE000227022A02B300B4006F0070009F01CBD0
:106ABE00019F02A002E200E900EA00B500B600B7AD
:106ACE0000CD008301CC008A0192019401210223A2
:106ADE000224022502260227022A02B300B4006F06
:0C6AEE000070009F01CB019F02A002007D
:00000001FF
